:020000040000FA
:100000000C9472030C949A030C949A030C949A0324
:100010000C949A030C949A030C949A030C949A03EC
:100020000C949A030C949A030C949A030C949A03DC
:100030000C949A030C949A030C949A030C949A03CC
:100040000C94D1260C949A030C949F260C94792638
:100050000C949A030C949A030C949A030C949A03AC
:100060000C941B270C949A0307634236B79BD8A7BE
:100070001A39685618AEBAAB558C1D3CB7CC5763CD
:10008000BD6DEDFD753EF6177231BF000000803F7B
:1000900008000000BE922449123EABAAAA2ABECD97
:1000A000CCCC4C3E00000080BEABAAAAAA3E000009
:1000B0000000BF000000803F000000000008417801
:1000C000D3BB4387D1133D190E3CC3BD4282AD2B38
:1000D0003E68EC8276BED98FE1A93E4C80EFFFBE30
:1000E00001C4FF7F3F00000000004E414E494E49D1
:1000F0005459494E46CDCCCC3D0AD7233C17B7D1F5
:100100003877CC2B329595E6241FB14F0A0000209A
:10011000410000C84200401C4620BCBE4CCA1B0E19
:100120005AAEC59D7400407A10F35A00A0724E1862
:10013000090010A5D4E80000E87648170000E40B99
:1001400054020000CA9A3B000000E1F5050000805F
:10015000969800000040420F000000A086010000B9
:1001600000102700000000E8030000000064000009
:100170000000000A00000000000100000000002C48
:1001800076D888DC674F0823DFC1DFAE59E1B1B70D
:1001900096E5E3E453C63AE651997696E8E6C284DA
:1001A00026EB898C9B62ED407C6FFCEFBC9C9F40F2
:1001B000F2BAA56FA5F490055A2AF75C936B6CF917
:1001C000676DC11BFCE0E40D47FEF520E6B500D0ED
:1001D000ED902E0300943577050080841E08000002
:1001E000204E0A000000C80C333333330F986E12D0
:1001F000831141EF8D2114893BE65516CFFEE6DBD6
:1002000018D1844B381BF77C1D901DA4BBE424201F
:100210003284725E228100C9F124ECA1E53D270001
:10022000000000230026002900FFE0FFD1AFFF32CD
:10023000FFD1FFFEFFE0FFD1AEFFD1FFFEFFE0FFE9
:10024000D11000FFFEFFD0FFE0FFC1FFD1AED5808F
:10025000A81FD300408D142002A1C8DA0281CFD993
:10026000F1DB402EA4A6AFFFD0FFFE005EBCE26132
:100270003FDD83C29C7E20A3FD1F41009D23BE461F
:10028000DB65F88C11AF32CA57E974000000002416
:100290000027002A0000000000250028002B000491
:1002A000040404040404040202020202020303031D
:1002B0000303030102040810204080010204081017
:1002C00020010204081020000000080002010000C4
:1002D000030407000000000000000001080D00FEFC
:1002E00009016102CD207FFE0BFE09FE0D00803268
:1002F000198980808080808080008028438390904E
:10030000901367874848FC48FC4848125989207870
:10031000A0A0702828F02012698944A44810102059
:10032000485488126787609090609488743813836B
:100330008080803239892040408080804040202267
:100340003989804040202020404080166585483013
:10035000FC30481455852020F8202011438370601C
:1003600080165181F821338340E0400279890202EE
:100370000408102040808012698930488484848475
:100380008448301259892060A02020202020F812B3
:1003900069897884840408304080FC126989FC04EF
:1003A0000810380404847812698908182848888855
:1003B000FC0808126989FC8080B8C404048478129F
:1003C000698938408080B8C4848478126989FC04C3
:1003D0000810102020404012698978848484788431
:1003E0008484781269897884848C74040408702168
:1003F000388840E040000040E040114888207020EC
:100400000000706080225989081020408040201030
:1004100008146484FC0000FC1259898040201008F4
:10042000102040801269897884840408101000101C
:100430001269897884849CA4AC948078126989308C
:1004400048848484FC848484126989F0888488F0D8
:10045000888488F01269897884808080808084789C
:10046000126989F088848484848488F0126989FC04
:10047000808080F0808080FC126989FC808080F020
:100480008080808012698978848080809C848C74CC
:1004900012698984848484FC84848484125989F850
:1004A00020202020202020F81279893E0808080802
:1004B00008088870126989848890A0C0A0908884F8
:1004C0001269898080808080808080FC02798982A6
:1004D00082C6AA92928282821269898484C4A49478
:1004E0008C84848412698978848484848484847864
:1004F000126989F8848484F880808080116A8A78FF
:100500008484848484A4947804126989F88484841B
:10051000F8A09088841269897884808078040484A3
:1005200078027989FE1010101010101010126989CD
:100530008484848484848484780279898282444493
:10054000442828281002798982828282929292AA73
:10055000440279898282442810284482820279895F
:10056000828244281010101010126989FC040810AF
:1005700020408080FC224989F080808080808080BB
:10058000F002798980804020100804020212498913
:10059000F010101010101010F01853832050880124
:1005A0007181FE3A2282804012668678047C848CB7
:1005B00074126989808080B8C48484C4B812668645
:1005C000788480808478126989040404748C84841B
:1005D0008C741266867884FC808478126989384429
:1005E0004040F840404040106888748888708078A7
:1005F0008478126989808080B8C484848484125885
:100600008820006020202020F8105A8A080018084E
:100610000808088888701269898080808890E09036
:1006200088841259896020202020202020F802761A
:1006300086EC9292929282126686B8C484848484F4
:10064000126686788484848478106888B8C484C4E8
:10065000B8808080106888748C848C7404040412C0
:100660006686B844404040401266867884601884AC
:10067000781268884040F8404040443812668688C6
:100680008888888874125686888888505020027618
:100690008682829292AA44126686844830304884C8
:1006A0001068888484848C74048478126686FC08BC
:1006B000102040FC22598938404020C0204040385A
:1006C000321989808080808080808080125989E002
:1006D00010102018201010E018538348A890FF0035
:1006E0003A28A62D11241FBECFEFD8E0DEBFCDBF24
:1006F00026E0A4E0B3E001C01D92AA34B207E1F7FE
:1007000013E0A0E0B1E0EAE9F5E702C005900D9240
:10071000A430B107D9F713E0C1E7D3E004C02197B3
:10072000FE010E943537C037D107C9F70E94C029A2
:100730000C94C03A0C940000089580E008958091D4
:100740000E0690910F06009739F120912106FC01C9
:10075000211123C03596E491E0932206FC013C96DA
:10076000E491E093230680912206082E000C990B59
:1007700020912306821B910927FD93952091240641
:10078000203441F0829FC001112426E09695879580
:100790002A95E1F7809325060895213039F43F9694
:1007A000E491E0932206FC017096DACF3D96E49145
:1007B000E0932206FC013E96D3CF08950895089554
:1007C000AF92BF92CF92DF92EF92FF920F931F935F
:1007D000CF93DF936C017B018B01040F151FEB019D
:1007E0005E01AE18BF08C017D10759F06991D60154
:1007F000ED91FC910190F081E02DC6010995892BC6
:1008000079F7C501DF91CF911F910F91FF90EF9084
:10081000DF90CF90BF90AF900895CF93DF93FC010E
:10082000448155816081718184E894E00E94E003F5
:10083000EC0142E050E066E671E084E894E00E945A
:10084000E0038C0F9D1FDF91CF910895FC01538D24
:10085000448D252F30E0842F90E0821B930B54179A
:1008600010F0CF96089501970895FC01918D828D27
:10087000981761F0A28DAE0FBF2FB11D5D968C91C0
:10088000928D9F5F9F73928F90E008958FEF9FEFFF
:100890000895FC01918D828D981731F0828DE80FBB
:1008A000F11D858D90E008958FEF9FEF0895FC0175
:1008B000918D228D892F90E0805C9F4F821B910942
:1008C0008F739927089584E894E00E94570421E0EB
:1008D000892B09F420E0822F089580E090E0892B95
:1008E00029F00E94630481110C9400000895FC011A
:1008F000A48DA80FB92FB11DA35ABF4F2C91848D81
:1009000090E001968F739927848FA689B7892C93DD
:10091000A089B1898C91837080648C93938D848D30
:10092000981306C00288F389E02D80818F7D808333
:100930000895EF92FF920F931F93CF93DF93EC01F3
:1009400081E0888F9B8D8C8D98131AC0E889F98976
:10095000808185FF15C09FB7F894EE89FF89608379
:10096000E889F98980818370806480839FBF81E0FA
:1009700090E0DF91CF911F910F91FF90EF9008953C
:10098000F62E0B8D10E00F5F1F4F0F731127E02E17
:100990008C8D8E110CC00FB607FCFACFE889F9894F
:1009A000808185FFF5CFCE010E947704F1CFEB8DDA
:1009B000EC0FFD2FF11DE35AFF4FF0829FB7F89423
:1009C0000B8FEA89FB8980818062CFCFCF93DF9341
:1009D000EC01888D8823B9F0AA89BB89E889F98957
:1009E0008C9185FD03C0808186FD0DC00FB607FC8C
:1009F000F7CF8C9185FFF2CF808185FFEDCFCE01BF
:100A00000E947704E9CFDF91CF91089590E0FC0137
:100A1000E953FD4F2491FC01ED54FD4F3491FC014D
:100A2000E156FD4FE491EE23C9F0222339F0233043
:100A300001F1A8F4213019F1223029F1F0E0EE0F94
:100A4000FF1FEB56FD4FA591B4918FB7F894EC9131
:100A5000611126C030953E233C938FBF0895273007
:100A6000A9F02830C9F0243049F7809180008F7DAB
:100A700003C0809180008F7780938000DFCF84B5A2
:100A80008F7784BDDBCF84B58F7DFBCF8091B000A5
:100A90008F778093B000D2CF8091B0008F7DF9CF57
:100AA0003E2BDACFCF93DF9390E0FC01ED54FD4F66
:100AB000249181569D4FFC0184918823D1F090E0D0
:100AC000880F991FFC01E557FD4FA591B491FC01DA
:100AD000EB56FD4FC591D49161110EC09FB7F894AC
:100AE0008C91E22FE0958E238C932881E223E8837A
:100AF0009FBFDF91CF9108958FB7F894EC91E22BCF
:100B0000EC938FBFF6CF8E3008F08E5020910E01FF
:100B100090E4299F900111248770822B80937C00A0
:100B200080917A00806480937A0080917A0086FDBB
:100B3000FCCF809178009091790008953FB7F894A8
:100B40008091FC039091FD03A091FE03B091FF03FF
:100B500026B5A89B05C02F3F19F00196A11DB11D18
:100B60003FBFBA2FA92F982F8827BC01CD01620F54
:100B7000711D811D911D42E0660F771F881F991F0F
:100B80004A95D1F708958F929F92AF92BF92CF92DC
:100B9000DF92EF92FF926B017C010E949E054B0158
:100BA0005C01C114D104E104F104B9F00E949E0576
:100BB000681979098A099B09683E73408105910586
:100BC00080F321E0C21AD108E108F10888EE880E0E
:100BD00083E0981EA11CB11CE4CFFF90EF90DF9042
:100BE000CF90BF90AF909F908F9008958F929F92DB
:100BF000AF92BF92CF92DF92EF92FF920F931F932B
:100C0000CF93DF938AE0A82EB12CD0E0C0E0EE2491
:100C1000EA9493E0F92E88248A9423E0922ED12C32
:100C2000C12C10E000E08FE00E948305081719072F
:100C300090F1C816D90608F46C018815990568F179
:100C40008E159F0508F47C01C80FD91F65E070E080
:100C500080E090E00E94C30581E0A81AB10819F76E
:100C60000C0D1D1DCE01801B910B8E199F0988193B
:100C7000990966E070E00E94CC36CB01DF91CF91FC
:100C80001F910F91FF90EF90DF90CF90BF90AF90AA
:100C90009F908F9008958C01D0CF4C01D5CF2FB766
:100CA000F8946091F8037091F9038091FA039091A0
:100CB000FB032FBF0895DC0180E0615090F09D910F
:100CC0009827E92FEF70F0E0E559FD4F2491E92FC7
:100CD000E295EF70F0E0E558FD4FE491822F8E270A
:100CE000ECCF0895DC012C911196ED91FC91F894D4
:100CF0008181822B81839281322F3095932392833D
:100D000087E090E00197F1F781818323818383E27B
:100D100090E00197F1F790817894EFECF0E0319753
:100D2000F1F7922381E009F480E00895FC019081BD
:100D30000180F281E02D292F209560FF14C0F894E6
:100D40008281822382838181892B8183A3E2B0E027
:100D50001197F1F78281982B9283789487ED90E038
:100D60000197F1F70895F89482818223828381812B
:100D7000892B8183AFEFB0E01197F1F78281982B37
:100D8000928378948FE090E0EBCFDF92EF92FF9226
:100D90000F931F93CF93DF93EC01D62EE42E08E040
:100DA00010E0FF24F39461E08D2D8F2109F460E0C1
:100DB000CE010E949606FF0C01501109A1F7E11027
:100DC00010C0F894E981FA81918188818095892306
:100DD0008183E981FA819281888180958923828348
:100DE0007894DF91CF911F910F91FF90EF90DF905A
:100DF0000895EF92FF920F931F93CF93DF938C018F
:100E00007B0140E065E50E94C506E70188E0E80E49
:100E1000F11C699140E0C8010E94C506CE15DF05AE
:100E2000C1F7DF91CF911F910F91FF90EF9008953F
:100E3000FC0190810180F281E02DF8948181292FBD
:100E400020958223818378943DE743E050E0315040
:100E500029F1DA011197F1F780818923C1F3F89420
:100E60008281822382838181892B81837894ABE77D
:100E7000B7E01197F1F7F894818182238183A3E190
:100E8000B1E01197F1F78081982381E009F080E0CB
:100E90007894E3E6F6E03197F1F7089580E008955D
:100EA0006F927F928F929F92AF92BF92CF92DF927A
:100EB000EF92FF920F931F93CF93DF93EC017B018F
:100EC0008A018E819F810E941807811102C090E0E3
:100ED00037C0B7018E819F810E94F90640E06EEB1A
:100EE0008E819F810E94C5067801680189E0C80E45
:100EF000D11CAE80BF8088E0882E912C712C662496
:100F00006394C5010E94720681117628660CE1E0A7
:100F10008E1A9108B1F7F70171927F01EC15FD056A
:100F200041F78E819F810E941807813081F668E029
:100F3000C8010E945B0691E0F80120852813C7CF05
:100F4000892FDF91CF911F910F91FF90EF90DF904C
:100F5000CF90BF90AF909F908F907F906F900895AB
:100F6000CF93DF93CDB7DEB729970FB6F894DEBFE6
:100F70000FBECDBFAE014F5F5F4F0E945007882369
:100F800031F08D818F33A9F020F48F31A1F080E012
:100F900007C08F3521F08F37D1F78CE001C08BE08F
:100FA00029960FB6F894DEBF0FBECDBFDF91CF916B
:100FB00008958AE0F5CF89E0F3CF2091D403260F7E
:100FC0003327331F21323105ECF420915A04FC0100
:100FD00090E080E0243069F082E00895A091D4038D
:100FE0002191AC014C545C4FA40FB52FB11D2C9333
:100FF0000196861798F38091D403680F6093D40309
:1010000080E0089581E0089510925A0481E0809371
:1010100059041092340461E082E10E94060561E007
:1010200083E10E940605E9EBF0E080818E7F8083FA
:1010300080818D7F808388E48093B80085E48093ED
:10104000BC000895CF93DF9391E09093B30388237E
:10105000B9F0C091B800D091BA008091BC008A7BF1
:101060008093BC0060E082E10E94060560E083E1BD
:101070000E9406050E940408D093BA00C093B800ED
:10108000DF91CF910895CF92DF92EF92FF920F936D
:101090001F93CF93DF93D091830481E0D13208F086
:1010A0009CC0C09182040E949E056B017C018091CE
:1010B0005A0481116CC082E080935A0481E08093CD
:1010C00059048FEF8093580410925704D09356041C
:1010D000A2E6B4E0E6E3F4E080E0D8138DC010921D
:1010E000350480913504CC0FC82BC0933504809112
:1010F0003404813009F084C0109234040E949E05AB
:101100006B017C01809135048093BB0080915C046D
:1011100090915D04A0915E04B0915F04892B8A2BAD
:101120008B2BA1F00E949E0500915C0410915D0440
:1011300020915E0430915F046C197D098E099F092E
:10114000061717072807390708F442C08091BC002A
:1011500083FDD8CF85EC8093BC000E949E056B0177
:101160007C0180915A04823009F44CC0809158046B
:101170008F3F09F469C080915804803209F466C039
:1011800080915804803309F463C084E026C08091C4
:101190005C0490915D04A0915E04B0915F04892B82
:1011A0008A2B8B2B09F483CF0E949E0500915C044F
:1011B00010915D0420915E0430915F046C197D09EB
:1011C0008E099F09061717072807390708F06FCF00
:1011D00080915B040E94220885E0109261041092C5
:1011E000830410926004DF91CF911F910F91FF90C3
:1011F000EF90DF90CF9008959D9191938F5F6DCF89
:1012000085EEA9CF80915C0490915D04A0915E046D
:10121000B0915F04892B8A2B8B2B09F4A2CF0E94FB
:101220009E0500915C0410915D0420915E04309154
:101230005F046C197D098E099F0906171707280797
:10124000390708F08ECFC4CF80E0C7CF82E0C5CF8A
:1012500083E0C3CFCF92DF92EF92FF920F931F9361
:10126000CF93DF93D82FC62F613208F098C00E9429
:101270009E056B017C0180915A0481116BC081E055
:1012800080935A04809359049FEF909358041092CE
:1012900057049C0F90935604809335048091350435
:1012A000DD0FD82BD093350480913404813009F0C0
:1012B00078C0109234040E949E056B017C018091DD
:1012C00035048093BB0080915C0490915D04A091F3
:1012D0005E04B0915F04892B8A2B8B2BA1F00E94B6
:1012E0009E0500915C0410915D0420915E04309194
:1012F0005F046C197D098E099F09061717072807D7
:10130000390708F448C08091BC0083FDD8CF85EC34
:101310008093BC000E949E056B017C0180915A0461
:10132000813009F440C0809157048C1710F4C091AB
:101330005704E6E3F4E0A4E1B4E080E08C1355C088
:101340008C2FDF91CF911F910F91FF90EF90DF9045
:10135000CF90089580915C0490915D04A0915E040B
:10136000B0915F04892B8A2B8B2B09F484CF0E94C8
:101370009E0500915C0410915D0420915E04309103
:101380005F046C197D098E099F0906171707280746
:10139000390708F070CF80915B040E942208C0E0FA
:1013A000CFCF85EEB5CF80915C0490915D04A09184
:1013B0005E04B0915F04892B8A2B8B2B09F4AECF8E
:1013C0000E949E0500915C0410915D0420915E04D2
:1013D00030915F046C197D098E099F090617170764
:1013E0002807390708F09ACFD6CF91919D938F5F48
:1013F000A5CF0895E091130480911204E81730F40A
:10140000F0E0EC5EFB4F808190E008958FEF9FEF5E
:10141000089590911304809112042FEF3FEF9817D5
:1014200048F4E92FF0E0EC5EFB4F208130E09F5F55
:1014300090931304C90108958091120490911304AC
:10144000891B990B0895CF92DF92EF92FF920F9331
:101450001F93CF93DF937C01CB018A01209160041D
:10146000222389F0EB016B01C40ED51ECC15DD05DE
:1014700069F06991D701ED91FC910190F081E02D27
:10148000C7010995F3CF642F0E94DD07C801DF91E2
:10149000CF911F910F91FF90EF90DF90CF90089523
:1014A000CF93DF931F92CDB7DEB76983209160049D
:1014B0002223F9F020918304203258F021E030E01B
:1014C000FC013383228390E080E00F90DF91CF9185
:1014D000089580916104E82FF0E0EE59FB4F998167
:1014E00090838F5F809361048093830481E090E018
:1014F000ECCF61E0CE0101960E94DD07F7CF80E0DE
:101500000895DC011696ED91FC91179712968C9137
:10151000481B477081E090E001C0880F4A95EAF7C8
:10152000E60FF11D3081222319F0832B808308956B
:1015300080958323FBCFFB014181DC0112962C9126
:101540001297421768F013962C911397241740F0C6
:10155000608115962C91621718F424810C94810AED
:101560000895FC0180819281980F928321819217C6
:1015700060F494819F5F94839381890F821710F0A8
:101580008FEF820F838381E0089580E00895FC014E
:10159000128280818150838314820895DB01ED9152
:1015A000FC910994CF93DF931F92CDB7DEB79E01D4
:1015B0002F5F3F4F47E40E94CE0A89810F90DF9151
:1015C000CF910895CF93DF931F92CDB7DEB79E01E1
:1015D0002F5F3F4F46E40E94CE0A89810F90DF9132
:1015E000CF910895BF92CF92DF92EF92FF920F9327
:1015F0001F93CF93DF938C01D42EE901FB01E2808E
:10160000F380F2E34F1709F476C0F417C8F08CE2C8
:10161000481709F470C0EDE24E17E9F0F7E14F17F3
:1016200079F19E014D2DB701C801DF91CF911F9136
:101630000F91FF90EF90DF90CF90BF900C94CE0A67
:1016400086E4481709F44CC0E7E44E1709F44EC08D
:10165000FBE34F13E6CFB701C8010E94D20AC9804D
:10166000C094C80EB701C8010E94E20A9881909503
:10167000890F8883C9828B818E5F83708B834BC077
:1016800047E1B701C8010E94CE0AB701C8010E9414
:10169000E20ABA80B094B80EB701C8010E94E20A0B
:1016A000D880D094D80EB701C8010E94D20ACB804E
:1016B000C094C80EB701C8010E94D20A99819095C2
:1016C000890FB882C982DA828B8381E0DF91CF9162
:1016D0001F910F91FF90EF90DF90CF90BF900895F2
:1016E000B701C8010E94E20A8883EFCFB701C801A1
:1016F0000E94D20AF9CFB701C8010E94D20AC9805C
:10170000C094C80EB701C8010E94E20A9881909562
:10171000890F8883C9829E014D2DB701C8010E949F
:10172000CE0AD3CFCF93DF93EC016A817B810E94F5
:10173000E20A88836A817B81CE010E94D20A898372
:101740006A817B8130E020E048E4CE010E94CE0A2D
:101750008B879E012D5C3F4F6A817B8147E1CE01E3
:10176000DF91CF910C94CE0ACF93DF93C0910C06FA
:10177000D0910D06E0913B06F0913C0682E0099580
:1017800030E020E04AE0BE018AE096E00E94CE0A06
:10179000C82FE0913B06F0913C0683E00995E0916B
:1017A0003B06F0913C0680E00995CC2329F08AE0C5
:1017B00096E00E94920BC1E08C2FDF91CF910895AB
:1017C000FC01808D8F5F08950B96FC018491089534
:1017D0000A96FC0184910895FC01849108950E9469
:1017E000EC0B882321F0823011F083E0089586E02D
:1017F0000895FC01E60FF11D849190E0982F882751
:101800003196E4918E0F911D089568E00C94F90BC8
:1018100066E00C94F90B5F926F927F928F929F9289
:10182000AF92BF92CF92DF92EF92FF920F931F93EE
:10183000CF93DF93EC01E62EF42EC22E0C811D8196
:10184000C8010E94EC0BD82E8C819D810E94EF0B69
:10185000982E21E0AA24AA94D21202C02FE0A22E30
:101860008C819D810E94E80BD82E8C819D810E94E5
:10187000E40BB82E8C819D810E94050CE0E6EC15EE
:1018800078F4009769F0080F191F91E6D92EBC145F
:10189000C0F4188A1B8A1C8A198A1A8A80E0A0C0A0
:1018A0008C819D810E94080CF0E4FC1538F40097AF
:1018B00029F0080F191F81E4D82EE9CF0F5E1F4FC2
:1018C000E6CFBD1430F3892D90E0F80124912F3F2D
:1018D00031F40F5F1F4FBD14E1F2D394F6CFCD105A
:1018E00072C08C819D810E94EC0B98012F5F3F4F4D
:1018F000F801882319F0823009F04EC084918B8B57
:10190000F90124912C8BF8013396E491E88BF801CE
:101910003496E491E98BF8013596E491EA8B011550
:10192000110509F4BBCF8C819D810E94EF0B3C898E
:10193000F31A9A89F91A9FEF930F9F0D2CA94EA9BC
:101940004F1508F449C0921718F49F1508F047C0C6
:101950002B899989E90E9FEF920F9E0D4BA95DA9E6
:101960005E1508F44DC0941718F49E1508F037C0A2
:10197000080F111D295F722E7694769476946F2C41
:10198000630E5E01FCE1AF0EB11C872C912CF614A6
:1019900031F15E2C68014AC08491982F9F7092505B
:1019A0009A8B82958F70898BF9012491822F8F7089
:1019B0008C8B22952F702B8BF8013296E491E29557
:1019C000EF70E88BACCF3296E491EA21E80FF92F63
:1019D000F11D0E0F1F1F7FCF921708F0B6CF888919
:1019E000DF91CF911F910F91FF90EF90DF90CF90FB
:1019F000BF90AF909F908F907F906F905F90089571
:101A0000941708F0B2CFEBCFF60184916A817B8105
:101A10005C8EFD8E1F8E8E8F95014BE3CE010E9452
:101A2000CE0AFFEFCF1ADF0A28E0520E8C2D801B62
:101A3000871550F3080D191DF394A9CF2EE93FE047
:101A4000009709F40895F9013197F1F70197F8CF5C
:101A5000CF93DF9300D0CDB7DEB720ED37E03A83E8
:101A600029839091BC00982311F081E00FC0298157
:101A70003A81232B81F48091110481FDF6CF80916E
:101A8000100481110DC091E0909310040F900F90FD
:101A9000DF91CF91089529813A8121503109DFCF1B
:101AA00080E0F4CF84EA8093BC0061E080E80E948B
:101AB000280D811102C080E008958091B900887FCF
:101AC000883051F0803141F0809110048111F3CFC2
:101AD00082E080931004EFCF88E78093BB0084E816
:101AE0008093BC0062E080E80E94280D882319F3EF
:101AF0008091110481FD05C08091B900887F8831F3
:101B000019F781E0089584E98093BC0064E080E1E6
:101B10000C94280D8093BB0084E88093BC0063E0A4
:101B200080E80E94280D8823A1F08091110481FD96
:101B30000DC08091B900887F883241F080911004F7
:101B4000811106C092E090931004089581E00895F9
:101B500080E008951092100408958093110410926B
:101B6000B90088E48093B8000C94AA0DCF93DF935A
:101B7000FC0123A5222389F0EC010E94520D811162
:101B800004C080E0DF91CF9108958EA1811107C03C
:101B90000E948A0D8823A9F31BA681E0F3CF80E47D
:101BA000F7CF0F931F93CF93DF93C62FD42F8901C5
:101BB000633001F138F4613099F0623009F449C0C2
:101BC000C1E012C0663029F1673091F16530C1F78C
:101BD0000E94B60D811117C00E94830DC0E004C0A1
:101BE000FC0186A50E94AD0D8C2FDF91CF911F9136
:101BF0000F910895FC0116A221E023A74111E0CF27
:101C00000E94830DDDCF8D2F0E948A0D8111D8CFC8
:101C1000E3CF0E94B60D8823F9F2DD2389F2F801A3
:101C200081918F010E948A0D8823B1F2D150F5CFA6
:101C30000E94B60D882381F2DD2311F2F801849110
:101C40000E948A0DC82F882379F20F5F1F4FD15051
:101C5000F3CFFC0146A321E023A7B2CFDB0114960A
:101C6000ED91FC9130E020E065E00994CF92DF92A5
:101C7000EF92FF920F931F93CF93DF938C017B0121
:101C80006A0180E0F601C491811110C081E0CF3F6C
:101C900049F04C2FB701C8010E942E0E882309F489
:101CA0004DC080E0BFEFCB1ADB0AECCF4FEFCF3F48
:101CB00089F3CE3F09F443C0C03F98F7C03E60F0BF
:101CC0004C2F4F70D7011496ED91FC9130E020E03D
:101CD00062E0C8010995E5CFC03D50F04C2F4F7030
:101CE000D7011496ED91FC9130E020E063E0F1CF54
:101CF000C03CF8F0D7011496ED91FC9130E020E063
:101D000040E064E0C8010995C295C07FCE5FD0E095
:101D1000CE010E941E0DD7011496ED91FC9130E08A
:101D200020E041E064E0C8010995CE010E941E0D4B
:101D3000B8CFC7FDB6CF8C2F90E0F8CF80E0DF9111
:101D4000CF911F910F91FF90EF90DF90CF9008956A
:101D5000AF92BF92CF92DF92FF920F931F93CF93D8
:101D6000DF936C018B01F42EE90180E1481709F43F
:101D700084C0841758F1AAE04A1709F462C0F80138
:101D800002811381F2E3FF1609F4CDC0FF1508F4B8
:101D90007FC085E1F81609F4CBC0A7E1FA1609F473
:101DA000DCC0B4E1FB126FC0D8011696ED91FC9136
:101DB000179715968C918E0F9F2F911D11928E174C
:101DC0009F07E1F7C8010E94C70A5DC0B1E14B1748
:101DD00009F45BC0E5E14E13D2CFFB01A280B380D2
:101DE0004DE352E0C6010E94360ED50114964C9187
:101DF000406BB801C6010E942E0ED8011496ED91D9
:101E0000FC9130E020E041E062E0C6010995F50177
:101E100026813781D8011496ED91FC91D501159654
:101E20004C9166E0C601099581111CC080E0DF91EC
:101E3000CF911F910F91FF90DF90CF90BF90AF9007
:101E40000895DB011496ED91FC9130E020E042E032
:101E500061E0C601099545E452E0B801C6010E945F
:101E6000360E8DCFD8011496ED91FC9130E020E034
:101E700040E063E0C601099582CF44E352E0B80137
:101E8000C6010E94360E81E0D2CF49E252E0F7CF80
:101E9000E6E4FE1609F46BC0F7E4FF1609F46CC023
:101EA0008BE3F812F0CF99818B8138E0390F8130C4
:101EB00031F0833011F0392F02C0392F985021E0D2
:101EC000D80113964C91491708F420E041E03917E6
:101ED00008F040E091E0F8015281351708F490E0F5
:101EE000322F342B932311F4242369F2FA80D12C5E
:101EF000C12C843048F490E0FC01EE5CFE4FC080C1
:101F0000825D9E4FDC01DC90F7FE04C0BE01C8017B
:101F10000E949B0A88818C0D888389818D0D89831D
:101F2000FF0C91F7B0CFBE01C8010E949B0AABCF56
:101F3000C8010E94B10A882309F478CFD801169607
:101F4000ED91FC91179715968C918E0F9F2F911DF7
:101F500011928E179F07E1F796CF1882F8018281C0
:101F60008983858181508A8383818B838CCFD8013B
:101F700015968C91888387CFF8018181FBCFDF9202
:101F8000EF92FF920F931F93CF93DF93EC01D62E26
:101F90001CAD0BAD7C0184E0E80EF11CE98DFA8DDF
:101FA000C7010995412F480F2D2D602FC7010E94B1
:101FB0000B0C9BAD890F8BAF81E090E0DF91CF914F
:101FC0001F910F91FF90EF90DF90089590E080E0D7
:101FD00008958F929F92AF92BF92CF92DF92EF922D
:101FE000FF92CF93DF93C8EDD5E0988121E0209355
:101FF0006004909382041092610410928304682F0D
:1020000081E295E00E94500A0E94430863E08881C3
:102010000E942A09109213048093120481E295E031
:102020000E94090A092E000CAA0BBB0B8824982ECB
:10203000A92EBA2E81E295E00E94090A092E000C11
:10204000AA0BBB0B6C017D01C828D928EA28FB2804
:10205000FE2CED2CDC2CCC2481E295E00E94090AB8
:10206000BC01990F880B990B6C297D298E299F291A
:10207000DF91CF91FF90EF90DF90CF90BF90AF9026
:102080009F908F9008958F929F92AF92BF92CF9220
:10209000DF92EF92FF920F931F932091E1052F3F64
:1020A00019F48AEF0E94E90F0091E5051091E60509
:1020B00030E020E0C72ED82EE92EFF24E7FCFA946A
:1020C000C01AD10AE20AF30A57E0959587957795E9
:1020D00067955A95D1F7000F111F221F331F4B012F
:1020E0005C01801A910AA20AB30AA5019401A09189
:1020F000E705B091E8050E943B374B015C01FBE02E
:10210000B594A79497948794FA95D1F7A70196016F
:10211000C701B6010E94BC369B01AC01ACE05595ED
:10212000479537952795AA95D1F7A091E905B091E4
:10213000EA050E943B379B01AC01BEE055954795EF
:1021400037952795BA95D1F7280D391D4A1D5B1D86
:102150002093DD053093DE054093DF055093E005C5
:10216000A5E0B0E00E94733360587F4F8F4F9F4FC0
:10217000672F782F892F992787FD9A950E943D32E6
:1021800020E030E048EC52E40E9431341F910F917E
:10219000FF90EF90DF90CF90BF90AF909F908F9087
:1021A00008952F923F924F925F926F927F928F92FB
:1021B0009F92AF92BF92CF92DF92EF92FF920F93D6
:1021C0001F93CF93DF93CDB7DEB76B970FB6F8941D
:1021D000DEBF0FBECDBF0E9443108091E1058F3F4F
:1021E00039F487EF0E94E90F6E8B7F8B888F998F70
:1021F0008091DD059091DE05A091DF05B091E005AD
:102200006C017D01FF0CCC08DC2C76019C01AD013A
:102210006C2D7C2D8C2D9C2D345F41405109610922
:1022200071098109910929873A874B87652E762E96
:10223000872E982E9B8F5901C42ED52EE62EF72E71
:10224000082F192F0E944337322E232E488B598B8B
:102250006A8B7B8B8C8B9D8B3091EE052091ED05ED
:10226000932F990F990B492F592F692F792F892F68
:102270000E9443370CE00E943B3829833C874A8FF9
:102280005D876E877F87582E492E3091F00520910B
:10229000EF05932F990F990BA32CB22CC888D988DE
:1022A000EA88FB880C891D89492F592F692F792FBE
:1022B000892F0E94433708E00E945438A980BC84CB
:1022C000CA8CDD84EE84FF84052D142D0E947138A4
:1022D00070588F4F9F4FE091EB05F091EC055F0137
:1022E000D12CC12CE12CF12C8701E983BA82CB825D
:1022F000DC82ED82FE820F831887C12CD12CE12C69
:10230000F12C00E010E00E94433701E20E945438B3
:102310002A8F532E49835C876D877E878F87492E4E
:10232000A0E00E94833809F436C13091F60520916F
:10233000F505932F990F990BA32CB22CC888D98837
:10234000EA88FB880C891D89492F592F692F792F1D
:10235000892F0E9443371901488B598B6A8B7B8BDD
:102360008C8B9D8B3091F4052091F305932F990F61
:10237000990BA984BA84CB84D62CE72CF82C092D90
:102380001B8D492F592F692F792F892F0E94433791
:1023900001E10E943B385101C888D988EA88FB884E
:1023A0000C891D890E94713859016A017B01382E00
:1023B000192F4E895F89688D798D84E075956795B1
:1023C000579547958A95D1F780E090E0A0E1B0E07D
:1023D000841B950BA60BB70B3C014D01990C6608AD
:1023E000762C43019C01AD01662D762D862D962D10
:1023F0000FE10E943B38722E832E942E5987B62F00
:10240000A72FF82FE92F3091F2052091F105932F96
:10241000990F990B492F592F692F792F892F03E293
:102420000E943B38032D0E94713859016A017B01DB
:102430008C01272D382D492D59856B2F7A2F8F2F01
:102440009E2F0E947A38E5E3AE2EFCE0BF2EC12C11
:10245000D12CE12CF12C00E010E00E944337AA8C33
:10246000B52CC980DC84ED84FE840F85142D0E9478
:102470009D372F873E8749875A876B8779838C875B
:102480009D870DE00E945438922E832E742E652E67
:10249000562E472E382E292E3091FC052091FB0513
:1024A000932F990F990BA92CB82CC72CD62CE52C5F
:1024B000F42C032D122D492F592F692F792F892F95
:1024C0000E9443370E94433709E10E945438AF8489
:1024D000BE84C984DA84EB84F9800C851D850E9452
:1024E000713819012A013B014C013091FA05209104
:1024F000F905932F990F990B492F592F692F792F90
:10250000892F0E94433703E10E94543859016A0120
:102510007B018C019101A201B301C4010E947138B9
:1025200008E00E94543859016A017B01E82F192FF5
:102530003091F8052091F705932F990F990B492FAA
:10254000592F692F792F892F04E00E943B380E2FD5
:102550000E9471380E94D93420E030E040E85BE30B
:102560000E949C326B960FB6F894DEBF0FBECDBFB3
:10257000DF91CF911F910F91FF90EF90DF90CF905F
:10258000BF90AF909F908F907F906F905F904F9093
:102590003F902F90089560E070E0CB01E3CFBF92B1
:1025A000CF92DF92EF92FF920F931F93CF93DF931F
:1025B000EC01B62EC72E8D85811105C0CE010E947B
:1025C000180781110EC01B861D861C8680E0DF91D6
:1025D000CF911F910F91FF90EF90DF90CF90BF9020
:1025E000089540E060EFCE010E94C50601E0E12CB5
:1025F000D12C11E0CE010E947206F82ECE010E946D
:10260000720691E0F91218C0813099F51134D8F2B0
:10261000DB86D11002C081E08D878B81882399F2FF
:102620002396EB2DFC2DCF01089629912193E817D5
:10263000F907D9F781E0CBCFEE2DF0E0F8120FC00B
:102640008B851817A0F4DE01AE0FBF1F13968C9177
:10265000802379F4F12C193008F41C87D12EEC0F6B
:10266000FD1F8381902F9095892383830AC0811356
:10267000F1CFFE01EE0DF11D8381802B8383FF24BA
:10268000F3946F2DCE010E9496061F5F000F11F488
:10269000E39401E087E08E1508F0ACCFB7CFDF926E
:1026A000EF92FF920F931F93CF93DF937C018B01E7
:1026B000D42EDC011696ED91FC91138615861486B6
:1026C0001286118610861782168215821482138252
:1026D000C0E0B801F701868197810E94CF12D82F00
:1026E000882329F0DC1629F0CF5FDC1690F7D0E0C4
:1026F00009C067E0C8010E945B06D80117969C914B
:102700008913F2CF8D2FDF91CF911F910F91FF9001
:10271000EF90DF900895CF939091E1059F3F41F5B1
:10272000682F8091D80591E0909360048093820493
:10273000109261041092830481E295E00E94500A95
:102740000E94430862E08091D8050E942A091092F5
:1027500013048093120481E295E00E94090AC82FB5
:1027600081E295E00E94090A20E03C2F282B392BBA
:10277000922F832FCF9108950F931F93CF93DF93C1
:10278000FC01048115810115110539F4FB0110824A
:10279000DF91CF911F910F9108954150510940173A
:1027A000510708F48A01EB01FC0160817181A801E5
:1027B000CE010E94973AC00FD11F1882E9CFCF9364
:1027C000DF93C091CC05D091CD05209761F0899120
:1027D000882349F0082E000C990B0E94713AFE01E3
:1027E00031978083F4CFDF91CF910895FC018081F0
:1027F0009181009711F00C94EC2D60E070E0CB011A
:102800000895FB0144815581FC0124813581241701
:10281000350778F080819181009759F0FB01608144
:1028200071816115710529F00E94893A21E0892B97
:1028300009F020E0822F08950F931F93CF93DF9329
:102840008C01EB01FC01808191810097E1F06881AE
:10285000798161157105A9F0428153812C813D81F7
:102860004217530770F00E94823A8C819D81F801D3
:10287000958384831D821C82DF91CF911F910F91DC
:1028800008950E942B3988819981F8019183808372
:102890008A819B81938382838C819D8195838483AC
:1028A000198218821B821A82E5CFCF93DF93EC0145
:1028B00088819981009711F00E942B391982188222
:1028C0001D821C821B821A82DF91CF910895FC0128
:1028D00080819181009711F00C942B3908950F930A
:1028E0001F93CF93DF93EC0188819981009759F072
:1028F0002A813B812617370730F081E0DF91CF91A5
:102900001F910F9108958B016F5F7F4F0E94B43923
:10291000009759F0998388831B830A832C813D811A
:10292000232B59F7FC011082E8CF80E0E7CFEF922C
:10293000FF920F931F93CF93DF936115710541F4BD
:1029400080E0DF91CF911F910F91FF90EF9008955C
:1029500041155105B1F07B01EC010C811D81040F83
:10296000151FB8010E946F14882351F32881398103
:102970008C819D81B701820F931F0E94823A1D8333
:102980000C8381E0DECF0F931F93CF93DF9300D0B2
:10299000CDB7DEB78C0169831A8241E050E0BE01F9
:1029A0006F5F7F4F0E949714811103C0C8010E947E
:1029B0005514C8010F900F90DF91CF911F910F9187
:1029C0000895CF93DF93EC01FB0101900020E9F71C
:1029D0003197AF01461B570B0E949714811103C01A
:1029E000CE010E945514CE01DF91CF910895CF936F
:1029F000DF93EC01FB0144815581608171810E946C
:102A00009714811103C0CE010E945514CE01DF91AD
:102A1000CF910895FB0144815581608171810C94AF
:102A20009714EF92FF920F931F93CF93DF93EC01D4
:102A30007B018A01BA010E946F1481110BC0CE0183
:102A40000E945514CE01DF91CF911F910F91FF90FD
:102A5000EF9008951D830C83B701888199810E94AE
:102A6000823AF0CFFB0101900020E9F73197AF01E6
:102A7000461B570B0C9411150F931F93CF93DF93A5
:102A8000CDB7DEB762970FB6F894DEBF0FBECDBFED
:102A90008C01CB01F80111821082138212821582FF
:102AA00014824AE0BE016F5F7F4F0E94132EBE0169
:102AB0006F5F7F4FC8010E94321562960FB6F8947F
:102AC000DEBF0FBECDBFDF91CF911F910F91089553
:102AD000CF93DF93EC01FB018617970749F06081E4
:102AE00071816115710541F0448155810E94111574
:102AF000CE01DF91CF9108950E945514F9CFFC01CA
:102B00001182108213821282158214820C9468152D
:102B1000FC011182108213821282158214826115C7
:102B2000710551F0FB0101900020E9F73197AF01E9
:102B3000461B570B0C9411150895AF92BF92CF927C
:102B4000DF92EF92FF920F931F93CF93DF936C016D
:102B50005B017A0189012417350720F48F2D790153
:102B6000042F182F68E671E0C6010E948815D50170
:102B70001496CD91DC91EC16FD06E0F40C171D07C0
:102B800008F4E801D501ED91FC911197EC0FFD1FC0
:102B9000108110826D917C916E0D7F1DC6016115B3
:102BA0007105A1F00E943215F50180819181C80F55
:102BB000D91F1883C601DF91CF911F910F91FF900C
:102BC000EF90DF90CF90BF90AF9008950E94551482
:102BD000EBCFCF93DF93EC01FB01248135810E9481
:102BE0009D15CE01DF91CF9108950F931F93CF9341
:102BF000DF93CDB7DEB72C970FB6F894DEBF0FBECC
:102C0000CDBFFC01248135811216130664F48C01BA
:102C1000253131059CF40E940D0464E170E080E0F0
:102C200090E00E94C3052C960FB6F894DEBF0FBE4D
:102C3000CDBFDF91CF911F910F9108952FE030E02C
:102C400050E040E0BC01CE0107960E949D154B85E7
:102C50005C856F81788584E894E00E94E00369E1F7
:102C600070E080E090E00E94C3054FE050E0B801C2
:102C7000CE0101960E94E915BE016F5F7F4FCE0124
:102C800007960E941C14CE0101960E946714CE0183
:102C900007960E940D0464E170E080E090E00E94DD
:102CA000C30568E671E0CE0107960E943215CE0199
:102CB00007960E946714B7CFEF92FF920F931F936E
:102CC000CF93DF93CDB7DEB7A1970FB6F894DEBFF1
:102CD0000FBECDBF7C01CB01BA01F701118210827A
:102CE000138212821582148242E0420F8E010F5F1E
:102CF0001F4F0E94CA2D009789F0BC01C7010E9496
:102D00003215A1960FB6F894DEBF0FBECDBFDF918E
:102D1000CF911F910F91FF90EF900895C7010E94EE
:102D20005514EFCF85ED8093BC0080915C049091A9
:102D30005D04A0915E04B0915F040796A11DB11DD2
:102D400023E0B695A795979587952A95D1F7209179
:102D5000BC0024FD03C010925A04089540915C0405
:102D600050915D0460915E0470915F04452B462B89
:102D7000472B69F30097A105B10541F025E32A959A
:102D8000F1F700000197A109B109E1CF80915B043F
:102D90000C9422080F931F93CF93DF93D62FC42F49
:102DA00010926A0110926901FC01448155814F5FC4
:102DB0005F4F21F069E671E00E94BC13E0911F06AD
:102DC000F09120068AE096E00995C80F09E611E027
:102DD000F80121918F01211105C0DF91CF911F9141
:102DE0000F9108954C2F6D2F8AE096E00E940B0CF6
:102DF000D80FEECF8F929F92AF92BF92CF92DF9279
:102E0000FF920F931F93CF93DF93CDB7DEB7AE97AB
:102E10000FB6F894DEBF0FBECDBF6C015B018A0117
:102E20000E944F061CA21BA21EA21DA218A61FA232
:102E300028EE33E040E050E00E941637CA01B901A5
:102E400020E831E541E050E00E9416372AE0AE016B
:102E50004F5F5F4F0E941E2EBE016F5F7F4FCE01FE
:102E600083960E943215BE016D5D7F4FCE010196A3
:102E70000E947F1569E972E0CE0101960E94E1147B
:102E8000BC01CE0189960E947F15CE0101960E9459
:102E90006714CE0183960E94671480910E0690916C
:102EA0000F068B5D924071F08BED92E090930F06D0
:102EB00080930E060E949F038DE993E09093200675
:102EC00080931F06109221060E949F0380EE9BE0D4
:102ED0009093200680931F0680911506803309F099
:102EE000B3C08FEF80932A0680932B068091430610
:102EF000811105C081E0809343060E94B40B80904D
:102F00000C0690900D06E0913B06F0913C0682E0A5
:102F10000995E0913B06F0913C0681E0099530E08F
:102F200020E044E1B4018AE096E00E94CE0A2DE35D
:102F300036E047E1B4018AE096E00E94CE0AE091D3
:102F40003B06F0913C0680E00995BE01675D7F4F2E
:102F5000CE0101960E947F1541E060E0CE0101960E
:102F60000E94CA16CE0101960E946714B601CE01D6
:102F700001960E947F1541E060E3CE0101960E9418
:102F8000CA16CE0101960E946714B501CE010196C2
:102F90000E947F1540E160E0CE0101960E94CA16B2
:102FA000CE0101960E946714E0911806F09119066F
:102FB000309719F08AE096E0099580900C06909081
:102FC0000D06E0913B06F0913C0682E00995E09108
:102FD0003B06F0913C0681E0099530E020E045E1B8
:102FE000B4018AE096E00E94CE0AF82E882341F0D0
:102FF0002DE336E047E1B4018AE096E00E94CE0A74
:10300000E0913B06F0913C0680E00995F1109DCFE0
:10301000B801110F880B990B0E94C305CE01899648
:103020000E946714AE960FB6F894DEBF0FBECDBFF8
:10303000DF91CF911F910F91FF90DF90CF90BF90C4
:10304000AF909F908F900895883231F0823031F0A8
:1030500081E080932A064ACF8FEFFBCF83E0F9CF40
:10306000FF920F931F93CF93DF93EC01F62E08810D
:103070001981C8010E945D33F81621F06F2DC80137
:103080000E946533CE01DF91CF911F910F91FF9088
:103090000895EF92FF920F931F93CF93DF9300D089
:1030A000CDB7DEB70DE215E08D5295407C01C7012A
:1030B000800F911F9A838983F80161918F01CE015E
:1030C00001960E943018F5E00B371F0781F78DE25B
:1030D00095E00F900F90DF91CF911F910F91FF908E
:1030E000EF900895EF92FF920F931F93CF93DF938A
:1030F00000D0CDB7DEB701E815E0815895407C01DE
:10310000C701800F911F9A838983F80161918F0114
:10311000CE0101960E943018F5E0083A1F0781F7AA
:1031200081E895E00F900F90DF91CF911F910F9163
:10313000FF90EF9008952F923F924F925F926F927F
:103140007F928F929F92AF92BF92CF92DF92EF9237
:10315000FF920F931F93CF93DF93CDB7DEB76E9798
:103160000FB6F894DEBF0FBECDBF60EC75E08CECFF
:1031700095E00E9468150E94DF1368E771E0CE01B8
:1031800001960E948815BE016F5F7F4F8CEC95E021
:103190000E940114182FCE0101960E94671411237A
:1031A00029F0F0E0E0E0099581E08EC06CE771E085
:1031B000CE0101960E948815BE016F5F7F4F8CEC97
:1031C00095E00E940114182FCE0101960E94671409
:1031D000112321F160E871E0CE0101960E9488156B
:1031E00068EA75E0CE0101960E94F714BC0182EDF9
:1031F00095E00E946815CE0101960E94671462ED69
:1032000075E0CE0101960E947F15CE0101960E94C5
:10321000F515CE0101960E946714C6CF6AE871E0E9
:10322000CE0101960E948815BE016F5F7F4F8CEC26
:1032300095E00E940114182FCE0101960E94671498
:10324000112369F06EE871E082ED95E00E9432157D
:103250006EEA75E082ED95E00E940A15D0CF6CE928
:1032600071E0CE0101960E948815BE016F5F7F4F0D
:103270008CEC95E00E940114182FCE0101960E945B
:1032800067141123D1F127E030E046E050E060EC14
:1032900075E0CE0101960E949D15BE016F5F7F4FC4
:1032A0008AEB95E00E941C14CE0101960E946714DF
:1032B0008AEB95E00E94F613672B19F4109206042E
:1032C00073CF81E0809306046E960FB6F894DEBF4C
:1032D0000FBECDBFDF91CF911F910F91FF90EF9067
:1032E000DF90CF90BF90AF909F908F907F906F9026
:1032F0005F904F903F902F90089563EA71E0CE0168
:1033000001960E948815BE016F5F7F4F8CEC95E09F
:103310000E940114182FCE0101960E9467141123F8
:1033200009F4BBC08091B1039091B203181619063D
:103330000CF03ACF88EC90E090930D0180930C0153
:1033400084E894E00E94E6041D861E861F86188A83
:10335000CC24C394D12C40EC242E43E0342E5E01C7
:10336000FDE0AF0EB11C2E0121E1420E511C51EBCC
:10337000652E53E0752E8091B1039091B2038C15A8
:103380009D050CF411CF80910C0190910D01813CB1
:10339000934024F030920D0120920C0100910C0119
:1033A00010910D01750148018A189B08C4018E0D0A
:1033B0009F1D0E945D33F70181937F01E415F505A0
:1033C000A9F7C801049690930D0180930C012DE894
:1033D000E22E23E0F22E09581340C8018E0D9F1DE6
:1033E0000E945D33F70181937F016E167F06A9F776
:1033F0004D855E856F85788923E0CE0107960E9412
:103400005C16BE01695F7F4FCE0101960E947F1559
:1034100067EA71E0CE0101960E94E114BC0182EDE1
:1034200095E00E946815CE0101960E946714CE01B6
:1034300007960E9467146DE873E0CE0101960E9422
:103440008815BE016F5F7F4F82ED95E00E940A15DF
:10345000CE0101960E94671462ED75E0CE010196DF
:103460000E947F15CE0101960E94F515CE010196AE
:103470000E94671480910C0190910D0184969093A5
:103480000D0180930C0164E170E080E090E00E9407
:10349000C305FFEFCF1ADF0A6ECF6AEA71E0CE01F3
:1034A00001960E948815BE016F5F7F4F8CEC95E0FE
:1034B0000E940114182FCE0101960E946714112357
:1034C000F1F126E030E045E050E060EC75E0CE013F
:1034D00001960E949D15BE016F5F7F4F8AEB95E0BC
:1034E0000E941C14CE0101960E9467148AEB95E09D
:1034F0000E94F613672B19F410928C0355CE81E0CD
:1035000080938C0388EC90E090930D0180930C01E4
:103510001092B2031092B1031092880310928903A3
:1035200010928A0310928B030E944F0660938403CB
:1035300070938503809386039093870335CE60EB69
:1035400071E0CE0101960E948815BE016F5F7F4F2A
:103550008CEC95E00E940114182FCE0101960E9478
:103560006714112309F479C08091C4059091C505B1
:10357000079708F419CE46E050E060EC75E0CE0104
:1035800001960E94E915BE016F5F7F4F8AEB95E0BF
:103590000E941C14CE0101960E9467148091BA0506
:1035A0009091BB05C12CD12C7601009721F00E948F
:1035B000E82D6B017C01C0921801D0921901E092B4
:1035C0001A01F0921B0167EB71E082ED95E00E9419
:1035D000321522E0B701A601CE0107960E945C16C3
:1035E000BE01695F7F4FCE0101960E947F1569E998
:1035F00072E0CE0101960E94E114BC0182ED95E0DB
:103600000E940A15CE0101960E946714CE0107960A
:103610000E94671462ED75E0CE0101960E947F154D
:10362000CE0101960E94F515CE0101960E94671405
:103630000E944F0628EE33E040E050E00E94F4364E
:10364000CA01B9010E943B3260930B0470930C04D1
:1036500080930D0490930E04A7CD62EC71E0CE012F
:1036600001960E948815BE016F5F7F4F8CEC95E03C
:103670000E940114182FCE0101960E946714112395
:1036800009F457C08091C4059091C505079708F4C7
:103690008BCD46E050E060EC75E0CE0101960E94D3
:1036A000E915BE016F5F7F4F8AEB95E00E941C1405
:1036B000CE0101960E9467148091BA059091BB05D6
:1036C000C12CD12C7601009721F00E94E82D6B01CE
:1036D0007C01C0920801D0920901E0920A01F092A7
:1036E0000B0169EC71E082ED95E00E94321521E05A
:1036F000B701A601CE0107960E945C16BE01695F64
:103700007F4FCE0101960E947F1569E972E0CE01DC
:1037100001960E94E114BC0182ED95E00E940A1519
:10372000CE0101960E946714CE0107960E9467148D
:1037300066CD64ED71E0CE0101960E948815BE0150
:103740006F5F7F4F8CEC95E00E940114182FCE0123
:1037500001960E9467141123D9F143E050E060EC18
:1037600075E0CE0101960E94E915BE016F5F7F4FA3
:103770008AEB95E00E941C14CE0101960E9467140A
:103780006AEB75E0CE0101960E947F1560E0CE01E4
:1037900001960E94C314BC018EEA95E00E94681550
:1037A000CE0101960E9467144091B2055091B30575
:1037B0004115510531F06FE275E08EEA95E00E9407
:1037C000BC1380911601909117010E944918ECCC0E
:1037D0006BED71E0CE0101960E948815BE016F5F0E
:1037E0007F4F8CEC95E00E940114182FCE010196BA
:1037F0000E946714112309F489C08091C405909137
:10380000C505409708F0D5C242E050E060EC75E095
:10381000CE0101960E94E915BE016F5F7F4F8AEBD2
:1038200095E00E941C14CE0101960E9467148091BD
:10383000BA059091BB05009709F441C00E94E82D9C
:1038400020E030E048EC52E40E949C320E94A33415
:103850006093390570933A0580933B0590933C053E
:1038600068ED71E082ED95E00E94321560913905B6
:1038700070913A0580913B0590913C058B019C012C
:1038800000591F452140310901341C4921053105EA
:10389000D0F06AEB75E0CE0101960E947F156EEDC7
:1038A00071E0CE0101960E94E114BC0182ED95E029
:1038B0000E940A15CE0101960E94671475CC60E043
:1038C00070E0CB01BDCF0E943D3220E030E048ECFB
:1038D00052E40E943134AB01BC0122E0CE010196DA
:1038E0000E945C16BE016F5F7F4F82ED95E00E94E3
:1038F0000A15CE0101960E94671443E050E06BEE7A
:1039000071E082ED95E00E9497145BCF6FEE71E05D
:10391000CE0101960E948815BE016F5F7F4F8CEC2F
:1039200095E00E940114182FCE0101960E946714A1
:103930001123F1F025E030E044E050E060EC75E068
:10394000CE0101960E949D15BE016F5F7F4F8AEBED
:1039500095E00E941C14CE0101960E9467148AEB28
:1039600095E00E94F61370937A056093790529CF4C
:1039700064EF71E0CE0101960E948815BE016F5F71
:103980007F4F8CEC95E00E940114182FCE01019618
:103990000E946714112309F45EC009E110E0C12CF4
:1039A000D12C760180E10E948305BC01990F880B20
:1039B000990B0E943D329B01AC01C701B6010E94E8
:1039C000C5336B017C016AE070E080E090E00E940A
:1039D000C3050150110931F720E030E040EA50E41E
:1039E000C701B6010E949C3220E030EC4FE754E45E
:1039F0000E94313420E030E048EC51E40E94313440
:103A0000609355057093560580935705909358051C
:103A100080911601909117010E94491868EF71E09A
:103A200082ED95E00E943215409155055091560562
:103A3000609157057091580522E0CE0107960E94CB
:103A40005C16BE01695F7F4FCE0101960E947F1513
:103A500060E072E05CCE63E072E0CE0101960E940D
:103A60008815BE016F5F7F4F8CEC95E00E940114BA
:103A7000182FCE0101960E946714112309F494CBEC
:103A800043E050E06CEC75E0CE0107960E94E9152A
:103A9000BE01695F7F4FCE0101960E947F1560E0F5
:103AA000CE0101960E94C314BC018AEB95E00E94EE
:103AB0006815CE0101960E946714CE0107960E94F8
:103AC00067146AEB75E0CE0149960E947F1567E0A6
:103AD00072E0CE0101960E9488158D8D9E8D892BF6
:103AE000C9F1098D1A8D69817A81C8010E94A63AAF
:103AF000009781F1FC01E01BF10B8F01CE010196D3
:103B00000E94671468E671E0CE0143960E94881512
:103B100068E671E0CE010D960E9488151016110618
:103B2000E4F469E072E0CE0101960E948815CE01AE
:103B300001960E94F515CE0101960E946714CE01F0
:103B40000D960E946714CE0143960E946714CE0121
:103B5000499661CB0FEF1FEFD1CFBE01675E7F4F5C
:103B6000CE010D960E946815D12CC12C8AEF682ECB
:103B700077247A9496E0592E89899A89009709F4D6
:103B800009C1F5E0CF16D104C9F36DEA72E0CE01A8
:103B900001960E948815BE016F5F7F4FCE010D9682
:103BA0000E940114182FCE0101960E946714111172
:103BB000CAC001E010E0980150E040E0BE01635F40
:103BC0007F4FCE0107960E949D15BE01695F7F4F12
:103BD000CE0101960E947F1560E0CE0101960E9401
:103BE000C314BC01CE0143960E946815CE01019614
:103BF0000E946714CE0107960E946714BE016D5E95
:103C00007F4FCE0107960E947F158B859C8502977A
:103C100008F49CC06DEA72E0CE0101960E948815FE
:103C2000BE016F5F7F4FCE0107960E940114F82EF0
:103C3000CE0101960E946714FF2009F487C022E09C
:103C400030E041E050E0BE01695F7F4FCE01019658
:103C50000E949D15CE0101960E94F6134B017B0137
:103C6000CE0101960E94671497FE03C02CE1E20E7C
:103C7000F11CB3016E197F095C9C70015D9CF00C16
:103C80001124F701EF57FA4F76876587CE01079623
:103C90000E946714B70166577A4F44E050E0CE01A6
:103CA00043960E94BC133FEFC31AD30A89899A89AD
:103CB0000817190708F067C0A801BE01635F7F4FAE
:103CC000CE0101960E94E915BE016F5F7F4FCE01C4
:103CD00043960E941C14CE0101960E946714BE01F7
:103CE0006D5E7F4FCE010D960E946815AD84BE8437
:103CF000A114B10409F440CF09891A89750101158D
:103D0000110509F439CF47014FEF841A940AF701DE
:103D10008081082E000C990B0E940532892BD9F462
:103D2000015011090A0D1B1DF8018081082E000C9D
:103D3000990B0E940532892B81F00E151F0568F042
:103D400001501109F1CF02E010E035CFCE01079606
:103D50000E94F61391CF7401D6CF0F5F1F4FA801B9
:103D60004E195F095A8B498BAE14BF0420F4B7017A
:103D7000C5010E94793AED85FE8589899A89E80F07
:103D8000F91F1082F9CE68E671E0CE010D960E940F
:103D90003215F2CEC0928305CC2041F081E08093B1
:103DA00081058EE190E00E947218C9CE10928105C3
:103DB000F8CF80E089CA2F923F924F925F926F9224
:103DC0007F928F929F92AF92BF92CF92DF92EF92AB
:103DD000FF920F931F93CF93DF93CDB7DEB7E99791
:103DE0000FB6F894DEBF0FBECDBF8C0168E671E060
:103DF00082ED95E00E943215C8010596059760F0A6
:103E000080910F04811108C00C3E2FEF120724F09F
:103E100010930A0400930904F8017A96E432F1053C
:103E200008F038C7EA5EF04E0C943537D7254A269D
:103E3000D3254A264A264A264A264A264A264A267A
:103E40004A26C920C920C9203A1F4B23C920C920AE
:103E50004E24C920C9205124602463244A26C92045
:103E6000C920C9207124C920A925C925C920C92074
:103E7000C920C92060E08FE00E945205E2ECF2E028
:103E8000E491ED8BEEEAF2E0E491F0E0EE0FFF1F3B
:103E9000E15EFD4F859194919F8B8E8B18A21AA2A3
:103EA00019A2CE01459698878F831D821E821982A2
:103EB00089E08A8381E08B838C831C8A1B8A1F8E16
:103EC0001E8E1D8E1C8E1B8E1A8E198E188E01E072
:103ED000BE016D5D7F4F8F8198850E94CF12882330
:103EE00009F45BC067E0CE0183960E945B069AA549
:103EF0008913EECF898181111DC08F8198850E9421
:103F00001807BE016D5D7F4F8F8198850E94F9066D
:103F100040E064EB8F8198850E94C5068F8198856B
:103F20000E947206182F8F8198850E941807111120
:103F300001C009831A818BA1803109F4B2C6BE0188
:103F40006D5D7F4FCE0101960E94B007811790F4FE
:103F50008A818A838D818F5F8D838BA1883231F036
:103F6000B0F4803119F0823209F0B2CF8E818F5FC8
:103F70008E83AECF8BA1803111F48CE0EACFBE01ED
:103F80006D5D7F4FCE0101960E94B007E2CF8B336B
:103F900069F3823409F09CCFE9CF8F8198850E9424
:103FA000180740E06CEC8F8198850E94C506498116
:103FB00064E48F8198850E94C5068B81882379F1FE
:103FC000EA81E9509EEEC92E92E0D92EE33038F412
:103FD000F0E0EE0FFF1FE85DFE4FC080D1808C81C6
:103FE000882309F461C0898181115EC00E944F0657
:103FF0004B015C010D2C000CEE08FF088F819885A9
:104000000E947206813059F00E944F066C197D099A
:104010008E099F09681579058A059B0578F38CE060
:104020008A83F12CE12C0FE5BFE7DB2E1FE1C12EC7
:104030008FE3B82E8D818E151F0409F00CF499C002
:104040004E2DBE01645D7F4FCE0101960E944F133D
:104050001A811D3080F11CE08CA5803181F1BE01F8
:10406000645D7F4FCE0101960E94B007181709F4D6
:1040700078C0AE014D5D5F4FBE01645D7F4FCE01E4
:1040800001960E945007882309F46BC08CA58031EB
:1040900009F467C01B3009F468C01C3091F01A3075
:1040A00009F065C0BFA20EC0B601DD0C880B990BEC
:1040B0000E94C305B4CF193078F619E0CDCF8CE05B
:1040C000D5CFDFA28F8198850E941807BE01645D5D
:1040D0007F4F8F8198850E94F90640E06EE48F81C2
:1040E00098850E94C50640E06DA18F8198850E9449
:1040F000C50640E06EA18F8198850E94C5068CA5FB
:10410000803131F040E06FA18F8198850E94C50613
:104110008F8198850E941807BE01645D7F4F8F8153
:1041200098850E94F906498168E48F8198850E94EC
:10413000C50664E170E080E090E00E94C3058981DB
:10414000882331F06AE070E080E090E00E94C305CF
:104150008F8198850E9418078A81811708F4812F22
:104160008A833FEFE31AF30A65CF0FA3ABCFCFA249
:10417000A9CF0E8110E0053011050CF0F2C0011539
:10418000110509F0F0C06BE775E082ED95E00E9443
:1041900068158091D6059091D705892B09F4C2C086
:1041A00062ED75E0CE0101960E947F15CE01019669
:1041B0000E94F515CE0101960E94671462ED75E02C
:1041C000CE0145960E947F1580918C03882309F4C7
:1041D000A5C08091B1039091B203843191050CF098
:1041E0009DC000910C0110910D01013CF3E01F07EF
:1041F0000CF094C001969093B2038093B1030E9497
:104200004F06C0908403D0908503E0908603F09021
:1042100087036C197D098E099F090E943B3220E0BB
:1042200030E04AE754E40E9431346093880370938D
:10423000890380938A0390938B03083C110534F41F
:1042400088EC90E090930D0180930C0180910C011B
:1042500090910D012CE8C22E23E0D22E08E813E045
:104260009C01285833407901C701800F911F9A8320
:104270008983D8016D918D01CE0101960E9430187D
:10428000C016D10689F7E0900C01F0900D01C7012E
:10429000049690930D0180930C01BE016B5E7F4FDD
:1042A000CE0101960E947F1560E0CE0101960E942A
:1042B000C314BC0182ED95E00E946815CE01019601
:1042C0000E9467144091D6055091D70541155105BC
:1042D00031F06DE873E082ED95E00E94BC130DE8CB
:1042E00013E0F701E958F3407F01C701800F911FE8
:1042F0009A838983D8016D918D01CE0101960E9428
:104300003018B3E0013B1B0781F780910C019091BD
:104310000D01849690930D0180930C01CE0145967A
:104320000E94671464E670E080E090E00E94C3059C
:10433000E9960FB6F894DEBF0FBECDBFDF91CF91E7
:104340001F910F91FF90EF90DF90CF90BF90AF90B3
:104350009F908F907F906F905F904F903F902F90A5
:10436000089504E010E068E671E082ED95E00E94B7
:104370003215A9E58A2EA5E09A2EB12CA12C4A2D42
:10438000BE01645D7F4FCE0101960E944F138111E3
:1043900051C0C12CD12CFEEFEF2EF2ECFF2EF40118
:1043A00041905190619071904F01A3019201C3011E
:1043B000B2010E948235811108C0A3019201C70198
:1043C000B6010E94C5336B017C01FFEFAF1ABF0A33
:1043D00020E030E04CEF52ECC701B6010E943632CB
:1043E00087FF74C0B501CE018C960E943C1565EA2A
:1043F00071E0CE0183960E948815BE01645D7F4FF7
:10440000CE0183960E94F7146AE971E00E94E114DC
:104410006BE775E00E94F714BC0182ED95E00E9405
:104420000A15CE0183960E946714CE018C960E94D5
:104430006714BDC0AE014D5D5F4FBE01645D7F4F2F
:10444000CE0101960E945007882309F4A2CF6CA1E7
:1044500070E0762F6627770F770F770F2BA148E054
:10446000249F90011124262B372B8CA58031D1F469
:104470006AA570E089A5DB01A81BB109CD0196955D
:10448000982F8827979587950E94E036CB01409713
:10449000B90153E0660F771F5A95E1F760789C01E8
:1044A000260F371F2138B4EE3B070CF472CFB90149
:1044B000330F880B990B0E943D3220E030E040E042
:1044C0005CE30E949C326B017C0169CF03301105D3
:1044D00009F4C2C0B501CE018C960E943C1565EA74
:1044E00071E0CE0183960E948815BE01645D7F4F06
:1044F000CE0183960E94F714BC0184EB95E00E94E4
:104500006815CE0183960E946714CE018C960E9496
:10451000671422E0B701A601CE018C960E945C16BA
:1045200064EB75E0CE0183960E947F1568E272E02D
:10453000CE0183960E94E114BE01645D7F4F0E940C
:10454000F714BC0184EB95E00E946815CE018396B8
:104550000E946714CE018C960E94671462ED75E08C
:10456000CE0183960E947F1564EB75E0CE018396A1
:104570000E94F714BC0182ED95E00E946815CE01FF
:1045800083960E94671462ED75E0CE0183960E94C7
:104590007F1560E2CE0183960E94C314BC0182EDB8
:1045A00095E00E946815CE0183960E9467140A1553
:1045B0001B0509F0E4CE03301105A9F460E272E0B6
:1045C000CE0183960E94881562ED75E0CE01839638
:1045D0000E94F714BC0182ED95E00E946815CE019F
:1045E00083960E9467146AE272E08AEB95E00E946B
:1045F000321562ED75E0CE018C960E947F156AEB54
:1046000075E0CE0183960E947F1544E650E0BE011E
:10461000645D7F4FCE0183960E94FA16CE01839689
:104620000E946714CE018C960E94671462ED75E0BB
:10463000CE0183960E947F1562E372E0CE018396DD
:104640000E94E114BC0182ED95E00E946815CE0144
:1046500083960E9467149DCD22E0B701A601CE018A
:1046600083960E945C16BE016D5D7F4FCE018C96D5
:104670000E947F1560E2CE018C960E94C314BC019B
:1046800082ED95E00E940A15CE018C960E94671477
:10469000CE018396CCCE60E080E10E9452058091ED
:1046A0000F048111F2C02AE030E040E050E02EAB70
:1046B0003FAB48AF59AF65E472E082ED95E00E94F0
:1046C0003215312C212C1CAA1DAAC12CD12C76010B
:1046D00002E310E0812C912C540180E10E948305BB
:1046E000092E000CAA0BBB0B880E991EAA1EBB1E1E
:1046F00065E070E080E090E00E94C3050150110980
:1047000061F74090550550905605609057057090A0
:104710005805C501B4010E943D3220E030E040EA76
:1047200050E40E949C3220E030E040E85AE30E94CE
:104730009C3220E030E048E452E40E943134A3018E
:1047400092010E94C43320E030E040E751E40E942F
:104750009C324B015C01A30192016AE979E989E38A
:1047600090E40E94C4339B01AC01C501B4010E94D6
:10477000313420E030E0A9010E94C53320E030E070
:1047800040E251E40E949C325B018C01232D322DCA
:104790004CA95DA90E942D35181624F43A2C2B2C17
:1047A0000CAB1DAB9FEFC91AD90AE90AF90A2EA969
:1047B0003FA948AD59AD2C153D054E055F050CF0E0
:1047C00087CF6EE170E080E090E00E94C3056CE46A
:1047D00072E082ED95E00E94321522E0432D522DC9
:1047E0006CA97DA9CE0101960E945C16BE016F5F87
:1047F0007F4FCE0145960E947F1569E572E0CE019C
:1048000045960E94E114BC018AEB95E00E94681570
:10481000CE0145960E946714CE0101960E9467144E
:1048200062ED75E0CE0145960E947F156AEB75E05A
:10483000CE0101960E947F1544E650E0BE016B5EFA
:104840007F4FCE0101960E94FA16CE0101960E947A
:104850006714CE0145960E94671460E672E0CE01AF
:1048600001960E9488156AEB75E0CE0101960E94C0
:10487000F71462ED75E00E94F714BC0182ED95E03B
:104880000E946815CE010196E4CE83E090E0A0E09E
:10489000B0E08EAB9FABA8AFB9AF0DCF0E944F0673
:1048A00078CC80910F04882321F082ED95E00E945E
:1048B0000D0468EC70E080E090E00E94C30569CCD4
:1048C00010920F0466CC81E080930F0480938905D9
:1048D0008091090490910A0490930804809307043E
:1048E00058CC80911501882309F453CC0E94D11033
:1048F0002B013C010E9443104B015C016091390582
:1049000070913A0580913B0590913C050E943D32A3
:1049100020E030E048EC52E40E9431346B017C012D
:104920000E94D11020E030E048EC52E40E94313483
:10493000A70196010E94313421E03EED42E45EE39E
:104940000E9432359B01AC0160E070E080E89FE39B
:104950000E94C43320E03AE24DE257E40E949C32C8
:104960006B017C0120E030E048EC52E4C301B2016D
:104970000E943134AB01BC0122E0CE0145960E9479
:104980005C16BE016B5E7F4FCE0101960E947F15C3
:1049900064E672E0CE0101960E94E114BC0184EB52
:1049A00095E00E946815CE0101960E946714CE0121
:1049B00045960E94671464EB75E08AEB95E00E94CF
:1049C00068156BED71E0CE0101960E94881564EBCD
:1049D00075E0CE0101960E94F714BC0184EB95E0CE
:1049E0000E946815CE0101960E94671421E0B5016E
:1049F000A401CE0145960E945C16BE016B5E7F4FFE
:104A0000CE0101960E947F1569E672E0CE01019603
:104A10000E94E114BC0182ED95E00E946815CE0170
:104A200001960E946714CE0145960E94671420E00B
:104A3000B701A601CE0145960E945C16BE016B5ED1
:104A40007F4FCE0101960E947F156CE672E0CE0189
:104A500001960E94E114BC018AEB95E00E940A15C0
:104A6000CE0101960E946714CE0145960E946714FC
:104A70006AEB75E0CE0101960E947F1562ED75E04C
:104A8000CE0145960E947F1544E650E0BE016F5F5F
:104A90007F4FCE0145960E94FA16CE0145960E94A0
:104AA0006714CE0101960E94671465ED71E0CE0196
:104AB00001960E94881562ED75E0CE0101960E9474
:104AC000F7146EE672E00E94E114BC0182ED95E0FD
:104AD0000E946815CE0101960E94671421E0B7017B
:104AE000A601CE0145960E945C16BE016B5E7F4F0B
:104AF000CE0101960E947F156CE672E0CE01019610
:104B00000E94E114BC0182ED95E00E940A15CE01DD
:104B100001960E946714CE0145960E94671464EBCB
:104B200075E0CE0101960E947F1562ED75E0CE0121
:104B300001960E94F714BC0182ED95E00E94681571
:104B4000CE0101960E94671465E070E080E090E07D
:104B5000B4CE81E080930E010E94F6058C0162E7DD
:104B600072E082ED95E00E94321560E074E0601B17
:104B7000710BCE0101960E943C15BE016F5F7F4F05
:104B800082ED95E00E940A15CE0101960E946714FD
:104B900000CB62E872E082ED95E00E9432150E943F
:104BA000F605BC01E6CFF0E0E0E00995F2CA80919D
:104BB000830518160CF055C081E0809381056DE8DF
:104BC00072E082ED95E00E94321580918105882384
:104BD00009F44AC06BE972E0CE0101960E94881583
:104BE00062ED75E0CE0101960E94F714BC0182EDE2
:104BF00095E00E946815CE0101960E94671462ED4F
:104C000075E0CE0101960E947F15CE0101960E94AB
:104C1000F515CE0101960E94671468EE73E080E0FE
:104C200090E00E94C3058091810581110E94552664
:104C300068E671E082ED95E00E94321580910F04E4
:104C4000809389058111A5CA6CEA72E086EC95E033
:104C50000E94321586EE9FEF90930A048093090418
:104C600098CA10928105ABCF63EA72E0CE0101963B
:104C70000E94881562ED75E0CE0101960E94F7143E
:104C8000BC0182ED95E00E946815CE0101960E945C
:104C90006714D4CF6FEA72E082ED95E00E9432157E
:104CA00078CA1D3008F054C968C90F931F93CF9379
:104CB000DF9301E815E0D0E0C0E00A5F1F4F80916C
:104CC0008305082E000C990BC817D9076CF4F8015E
:104CD000878190850E94DB1E68EE73E080E090E0A3
:104CE0000E94C3052196E9CFDF91CF911F910F91CB
:104CF00008951F920F920FB60F9211242F933F9396
:104D00004F935F936F937F938F939F93AF93BF93D3
:104D1000EF93FF9384E894E00E947704FF91EF9172
:104D2000BF91AF919F918F917F916F915F914F91C3
:104D30003F912F910F900FBE0F901F9018951F92CB
:104D40000F920FB60F9211242F938F939F93EF938F
:104D5000FF93E0919404F09195048081E0919A048E
:104D6000F0919B0482FD1BC0908180919D048F5F18
:104D70008F7320919E04821741F0E0919D04F0E032
:104D8000EC57FB4F958F80939D04FF91EF919F917E
:104D90008F912F910F900FBE0F901F9018958081CB
:104DA000F4CF1F920F920FB60F9211242F933F93BF
:104DB0008F939F93AF93BF938091F8039091F903E2
:104DC000A091FA03B091FB033091F70323E0230F86
:104DD0002D3758F50196A11DB11D2093F70380933F
:104DE000F8039093F903A093FA03B093FB03809127
:104DF000FC039091FD03A091FE03B091FF03019687
:104E0000A11DB11D8093FC039093FD03A093FE03AD
:104E1000B093FF03BF91AF919F918F913F912F91DD
:104E20000F900FBE0F901F90189526E8230F029643
:104E3000A11DB11DD2CF1F920F920FB60F92112458
:104E40002F933F934F935F936F937F938F939F9392
:104E5000AF93BF93EF93FF938091B900887F803623
:104E600009F44AC0F0F5883209F4A7C018F580317A
:104E700009F49BC0B8F4882309F4F9C0883009F418
:104E800094C0FF91EF91BF91AF919F918F917F91CE
:104E90006F915F914F913F912F910F900FBE0F90A7
:104EA0001F901895883109F488C0803251F780939B
:104EB000580414C0803409F49DC040F48033B9F321
:104EC0008833F9F68093580485ECB0C0803509F436
:104ED00085C0883509F496C0883499F60E949216E8
:104EE000D0CF883909F48CC038F5883729F050F4D0
:104EF000883611F0803729F683E080935A041092A7
:104F0000F60357C0883809F47BC0803919F080381F
:104F100009F0B7CF8091F603803208F071C0E091BC
:104F2000F60381E08E0F8093F6038091BB00F0E0E2
:104F3000EA52FC4F80833DC0803B39F0E0F4803A78
:104F400009F479C0883A09F09CCF84E080935A0430
:104F50001092D5031092D403E0910204F09103045F
:104F600009958091D40381110FC081E08093D4030F
:104F70001092B40309C0803C09F4A6CF883C09F420
:104F8000A3CF883B09F07DCFE091D50381E08E0F60
:104F90008093D503F0E0EC54FC4F80818093BB00FC
:104FA0009091D5038091D40329C0809135048093DA
:104FB000BB0085EC8093BC0064CF90915704809136
:104FC0005604981758F5E091570481E08E0F8093AE
:104FD0005704F0E0EA5CFB4F8081E9CFE091570491
:104FE00081E08E0F809357048091BB00F0E0EA5C73
:104FF000FB4F808390915704809156049817C8F214
:1050000085E8D8CFE091570481E08E0F8093570454
:105010008091BB00F0E0EA5CFB4F808380915904F3
:1050200081115CCF81E08093340484EA8093BC00DA
:1050300010925A0426CF85EC8093BC0010925A043B
:105040008091F603803230F4E091F603F0E0EA520A
:10505000FC4F10826091F60370E0E0910004F09143
:10506000010486ED93E009951092F6030ACF1092A1
:10507000580434CFCF93DF931092870410928604A4
:1050800088EE93E0A0E0B0E08093880490938904D8
:10509000A0938A04B0938B042AE331E03093850413
:1050A0002093840425EC30E0309391042093900405
:1050B00024EC30E0309393042093920420EC30E011
:1050C000309395042093940421EC30E030939704BE
:1050D0002093960422EC30E03093990420939804B6
:1050E00026EC30E030939B0420939A0410929D04A8
:1050F00010929E0410929F041092A0041092240516
:10510000109223058093250590932605A0932705EB
:10511000B09328058CE491E09093220580932105BB
:1051200010920906109208068EE591E0909307060A
:105130008093060610924106109242061092430692
:1051400010920F0610920E06109211061092100681
:105150001092130681E08093120682E28093140677
:105160001092190610921806EDE2F6E08BE396E035
:10517000CFEFC1938E179F07E1F7D1E0D0932A06B6
:105180008DE993E09093200680931F06D09321062B
:10519000109222061092230680E480932406109237
:1051A00025068CE993E090933C0680933B068CE1C6
:1051B00091E090930D0680930C06109238060E94A1
:1051C000B40B8EE591E09093070680930606C0939A
:1051D000E105C093E205C093E305C093E40568E6EA
:1051E00071E082ED95E00E94881568E671E08CEC34
:1051F00095E00E94881568E671E086EC95E00E94D3
:10520000881568E671E080EC95E00E94881568E6F4
:1052100071E08AEB95E00E94881568E671E084EB06
:1052200095E00E9488156DEB72E08EEA95E00E9491
:10523000881564EC72E088EA95E00E948815109267
:10524000810585E080938205109283051092850583
:105250001092840510928705109286051092880599
:105260001092890561ED72E08BE795E00E94881548
:1052700086E190E090932E0580932D058CE79CE8C5
:10528000A1E0B0E08093390590933A05A0933B05E7
:10529000B0933C0581EA97E6A3E3BDEB80933D051F
:1052A00090933E05A0933F05B093400586E696E6B1
:1052B000A6EABFE38093410590934205A09343057E
:1052C000B09344051092450510924605109247058B
:1052D000109248051092490510924A0510924B050C
:1052E00010924C05D0934D0589E190E090934F05C5
:1052F00080934E05D093500580E090E4ACE1B5E496
:105300008093510590935205A0935305B093540593
:105310001092550510925605109257051092580597
:10532000E9E5F5E080E1DF011D928A95E9F7109249
:10533000690510926A0510926B0510926C05109227
:105340006D0510926E0510926F0510927005109207
:1053500071051092720510927305109274051092E7
:10536000750510927605109277051092780581E008
:1053700090E090937A0580937905DF91CF9108951D
:10538000CF93DF93CDB7DEB72C970FB6F894DEBF7F
:105390000FBECDBF789484B5826084BD84B5816032
:1053A00084BD85B5826085BD85B5816085BD8091F0
:1053B0006E00816080936E00109281008091810068
:1053C0008260809381008091810081608093810060
:1053D000809180008160809380008091B100846022
:1053E0008093B1008091B00081608093B000809183
:1053F0007A00846080937A0080917A008260809342
:105400007A0080917A00816080937A0080917A009E
:10541000806880937A001092C10061E08EE00E9463
:105420005205E0919404F091950482E08083E0912C
:105430009004F09191041082E0919204F091930411
:105440008FEC808310929C04E0919804F091990471
:1054500086E08083E0919604F091970480818061DA
:105460008083E0919604F091970480818860808326
:10547000E0919604F0919704808180688083E091A8
:105480009604F091970480818F7D808360E08EE0A8
:105490000E94060568EC70E080E090E00E94C30581
:1054A00084E690E090931701809316010E945D338B
:1054B0008093040485E690E00E945D3380930504A8
:1054C0000091040410910504B801012E000C880B12
:1054D000990B0E943D329B01AC010E9482358111E3
:1054E00006C00B5011090C30110508F45FC184E6A9
:1054F00090E00E94491831E8C32E35E0D32E5601C2
:105500000EE110E0C8010E945D33F50181935F0157
:105510000F5F1F4F07321105A9F710918205612F08
:10552000012E000C770B880B990B0E943D329B01DA
:10553000AC010E948235811103C0153009F459C1B4
:105540008EE190E00E94721868EC70E080E090E0DC
:105550000E94C3056DED72E082ED95E00E94321568
:10556000109213041092120410926104109283049A
:105570000E9404088DED93E090930304809302044D
:105580008EED93E0909301048093000464E670E054
:1055900080E090E00E94C30569E671E0CE010196CB
:1055A0000E948815CE0101960E94F515CE01019644
:1055B0000E94671480910C0690910D06F1E08F30E7
:1055C0009F0751F090931201809311018FE091E0B9
:1055D00090930D0680930C0682EF9AE09093100151
:1055E00080930F018AE096E00E94920B62ED75E0D5
:1055F000CE0101960E947F156EEA75E0CE010796F6
:105600000E947F1548EE53E0BE016F5F7F4FCE01D1
:1056100007960E94FA16CE0107960E946714CE01E3
:1056200001960E9467146EEA75E0CE0101960E9411
:105630007F1560E0CE0101960E94C314BC0182ED8B
:1056400095E00E940A15CE0101960E94671462ED52
:1056500075E0CE0101960E947F15CE0101960E9451
:10566000F515CE0101960E94671486E78093D80550
:105670008091E1058F3FB1F410921304109212044F
:1056800010926104109283040E9404088DED93E04F
:1056900090930304809302048EED93E090930104B1
:1056A000809300048091E1058F3F01F58091D8053A
:1056B00091E09093600480938204109261041092B0
:1056C000830460ED81E295E00E94500A0E94430845
:1056D00061E08091D8050E942A09109213048093FA
:1056E000120481E295E00E94090AF82E28E5F216DC
:1056F00009F48DC066EE72E082ED95E00E943215ED
:105700001092150162ED75E0CE0101960E947F15A1
:10571000CE0101960E94F515CE0101960E946714F4
:105720008AE2C82ED12C98EE892E93E0992EA12CD6
:10573000B12C20E0E22E20E0F22E01E068E671E0DC
:10574000CE0107960E94881510E084E894E00E943C
:105750005704181619060CF0CBC01111C9C084E803
:1057600094E00E9435048A3009F072C11091060459
:10577000112309F482C18091C4059091C505892B3C
:1057800009F474C162EF72E0CE0101960E9488159F
:10579000BE01695F7F4FCE0101960E94F7140E94FF
:1057A0000D04CE0101960E94671460C14DE2C42E23
:1057B00045E0D42E04E610E0C8010E945D33F601F6
:1057C00081936F010F5F1F4F023B1105A9F76FE235
:1057D00075E0CE0101960E948815BE016F5F7F4F74
:1057E0008EEA95E00E941C14CE0101960E94671477
:1057F00082CE0EE110E0C8010E945D33F601819374
:105800006F010F5F1F4F05341105A9F79DCE88E882
:105810000E948B139093E6058093E5058AE80E9429
:105820008B139093E8058093E7058CE80E948B1317
:105830009093EA058093E9058EE80E948B1390937C
:10584000EC058093EB0580E90E948B139093EE05A5
:105850008093ED0582E90E948B139093F00580936D
:10586000EF0584E90E948B139093F2058093F10574
:1058700086E90E948B139093F4058093F30588E9E1
:105880000E948B139093F6058093F5058AE90E9498
:105890008B139093F8058093F7058CE90E948B1386
:1058A0009093FA058093F9058EE90E948B139093EB
:1058B000FC058093FB058091E1058F3F09F030CF17
:1058C0008091D80591E090936004809382041092B7
:1058D00061041092830464EF81E295E00E94500A13
:1058E0006FE381E295E00E94500A0E94430818CFBE
:1058F0008B859C85892B51F084E894E00E94E60416
:1059000064E170E080E090E00E94C305BE01695F41
:105910007F4F80EC95E00E941C14CE0107960E94F8
:10592000671468E671E082ED95E00E94321580917F
:10593000C4059091C5058130910509F0C6C060ECA1
:1059400075E08CEC95E00E9468150E94DF136CEC0A
:1059500075E0CE0101960E947F158D819E81892B75
:1059600009F4A5C0E981FA81309709F4A0C08081CB
:10597000823409F484C0833409F48EC0813409F080
:1059800096C06BEF72E080EC95E00E943215CE017C
:1059900001960E94671480EC95E00E94F613CB01FB
:1059A0000E94DB1E80910F04882309F43FC00E94EF
:1059B0004F06A50194010E94F436CA01B9010E9464
:1059C0003B3220910B0430910C0440910D04509116
:1059D0000E040E94C43320911801309119014091A6
:1059E0001A0150911B010E942D351816FCF480916C
:1059F000090490910A044A9609F4A0C08091070412
:105A0000909108040E94DB1E0E944F06A50194019C
:105A10000E94F436CA01B9010E943B3260930B0424
:105A200070930C0480930D0490930E046AE070E070
:105A300080E090E00E94C305E114F10409F47ECEF9
:105A40000E946304882309F479CE0E94000076CE78
:105A50008D3009F48BCE89831A8241E050E0BE017B
:105A60006F5F7F4FCE0107960E9497146AE070E047
:105A700080E090E00E94C30568CE11E0F7CF6EEFA2
:105A800072E080EC95E00E94321510920F048CEFCA
:105A90009FEF0E94DB1E7BCF61E073E080EC95E01E
:105AA0000E94321500930F048DEF9FEFF2CFBE01DD
:105AB0006F5F7F4F80EC95E00E9468156AE070E0B0
:105AC00080E090E00E94C30562CF049768F56DEA1C
:105AD00072E0CE0101960E948815BE016F5F7F4F74
:105AE00080EC95E00E940114182FCE0101960E94CF
:105AF00067141123C9F08091C4059091C5050297E0
:105B000088F0E091C005F091C105309759F081818E
:105B100080330CF4845EF601E81BF10987FDF395F0
:105B2000CF013ECF80E0F6CF8091C4059091C505AE
:105B3000029708F437CF0E949B1834CF80918105DB
:105B4000882309F461CF0E9455265ECF8BE795E04C
:105B50000E94671488EA95E00E9467148EEA95E037
:105B60000E94671484EB95E00E9467148AEB95E02D
:105B70000E94671480EC95E00E94671486EC95E023
:105B80000E9467148CEC95E00E94671482ED95E00A
:105B90000C946714EF920F931F93CF93DF93E80158
:105BA00034E047FD34E1042E000C550B57FF03C0D1
:105BB000519541955109E32E022F242FAE010E94E9
:105BC0007E2ECE01DF91CF911F910F91EF9008951E
:105BD000662777270C94DD2F1F93FC0199278827D0
:105BE000BC01E89411911032E9F3193010F01E3025
:105BF000C8F31B3251F01D3249F4689406C00E946C
:105C00002D2E610F711D811D911D119110531A30A0
:105C1000B0F33EF490958095709561957F4F8F4FCE
:105C20009F4F1F910895BB274A3031F4992322F4E6
:105C3000BDE2909581959F4F0C94652EBB272A302D
:105C400051F4992342F4BDE2909580957095619549
:105C50007F4F8F4F9F4F0C94432E592F482F372F34
:105C6000262F660F771F881F991F660F771F881FC3
:105C7000991F620F731F841F951F660F771F881F60
:105C8000991F0895BB27FA01A62F62177105810598
:105C90009105330B30FB66F0AA27660F771F881F2C
:105CA000991FAA1FA21710F0A21B63953850A9F7DD
:105CB000A05DAA3308F0A95DA19336F7B111B193A5
:105CC0001082CA010C942632BB27FB015527AA2754
:105CD000880F991FAA1FA41710F0A41B8395505179
:105CE000B9F7A05DAA3308F0A95DA193009779F7F1
:105CF000B111B1931192CB010C942632A9E0B0E01E
:105D0000E4E8FEE20C9484336A01F22EB02E102FE8
:105D1000FBE3AF2EA01608F41BE31F5F012F27E063
:105D2000AE014F5F5F4F0E942D31BC018981982FDA
:105D30009970913009F43FC09BE2E1FC04C09E2DB4
:105D40009170E0FC3AC05E2D5071E82FE87083FF3F
:105D500046C084E0911101C083E0EF2DE81B8F1550
:105D600008F0E0E0D6018E2F20E2552351F199236F
:105D700029F0D6019C93C60101966C0196012D5F16
:105D80003F4FE2FE24C08EE4D6018C9391E411963D
:105D90009C93119712968C93D9018E2F90E28111CA
:105DA0001BC0E20FF32FF11D10828EEF9FEF29969B
:105DB000ECE00C94A0339DE2C6CF90E2C4CF2D93CB
:105DC00081508111FCCFCE0ED11CE0E0D0CF8EE609
:105DD000D6018C9391E6DBCF9D938150E0CF482F85
:105DE000447082FF3DC084E0911101C083E08F15B3
:105DF00010F4EF2DE81BD6018E2F20E2552309F178
:105E0000992329F0D6019C93C60101966C01960155
:105E10002D5F3F4FE2FE1BC089E4D6018C938EE4D8
:105E200011968C93119786E412968C93D9018E2F3C
:105E300090E2882309F4B5CF9D938150FACF2D933A
:105E400081508111FCCFCE0ED11CE0E0D9CF89E684
:105E5000D6018C938EE611968C93119786E6E4CF4B
:105E60009B0177FF02C030E020E0A1E0B0E091119B
:105E700002C0B0E0A0E0F9013196AE0FBF1F8B2C3D
:105E8000912CBB2009F461C05401EFEFAE1ABE0A99
:105E9000AA0DBB1DFA161B0619F014F04F2D4A1B54
:105EA000511188C0E3FC59C07601A42FB0E2A111C2
:105EB0004FC0C40ED11C992309F45BC040E0D60149
:105EC0001196F60190836D01552309F448C0012F06
:105ED000060F9A81582F507184FF03C0913309F443
:105EE000015010160CF047C0093008F008E0EEE24F
:105EF000FE2E5B01A01AB10885019194819491084E
:105F00002F3F320729F4D601FC92F60131966F013A
:105F10006217730794F1021713077CF5DB01A21BCC
:105F2000B30BAA24A394B12CAC0EBD1EAA0DBB1DAD
:105F300011968C9121503109D601119628153905F9
:105F4000F4F0F60180836D01DBCFB12CA12CA0CF42
:105F5000F701B1937F01A150AACF9111B0CFD60123
:105F6000942F50E302C05D9391509111FCCFC40E69
:105F7000D11C40E0ACCF01E0BACF80E3DBCF6217A9
:105F8000730731F4963388F4953311F4552369F08F
:105F9000F6018083FD01842F90E2811108C0A40FD7
:105FA000B11D1C9290E080E002CF81E3F1CF91938C
:105FB0008150F3CF911183CF8ACFB0E0A0E0E3EE20
:105FC000FFE20C9484335C017B016115710519F0CB
:105FD000DB018D939C9385010F5F1F4FF501D081ED
:105FE0008D2F90E00E9405326C01892BB9F5DD32CE
:105FF000B9F50F5F1F4FD5011196DC91C1E0580133
:10600000F1E0AF1AB10843E050E062EF70E0C50183
:106010000E940E32892B69F5680182E0C80ED11CFE
:1060200045E050E06DEE70E0C6010E940E32892B13
:1060300021F4680197E0C90ED11CE114F10419F0B4
:10604000D701CD92DC9260E070E080E89FEFC11153
:10605000FFC060E070E080E89FE7FAC05801BBCF66
:10606000DB3229F485010E5F1F4FF501D181C0E0BD
:10607000C6CF43E050E06AEE70E0C5010E940E32E8
:10608000892BE9F0F80110E000E020E030E0A90100
:106090005F01B0ED8B2E8D0E89E08815C8F19C2E26
:1060A000689491F88C2F8870C2FF16C0811102C0CD
:1060B0000F5F1F4F3196D501DC91C92DE9CFE11457
:1060C000F10429F00E5F1F4FF7011183008360E098
:1060D00070E080EC9FE7BCC0882311F001501109EB
:1060E000A5E0B0E00E9473339B01AC01220F331F87
:1060F000441F551F280D311D411D511D283999E997
:106100003907490799E15907A8F2C6609C2ED2CFFA
:10611000AEEF8A1206C0C3FD3CC09C2E689493F873
:10612000C9CFDF7DD534A9F580818D3239F4C061C6
:10613000DF011296818162E070E006C0DF018B32E0
:10614000C1F3119661E070E080535D01A61AB70AB1
:106150008A30F8F4E0E8CE16ECE0DE065CF4B60136
:10616000660F771F660F771FC60ED71ECC0CDD1C7F
:10617000C80ED11C5D01FFEFAF1ABF0A8C9180538E
:106180008A30A8F1C4FF03C0D194C194D1080C0D8A
:106190001D1DC1FF09C0E114F10431F081E0A81A0E
:1061A000B108D701AD92BC92CA01B9010E943B323D
:1061B000C370C33009F490584B015C0120E030E01B
:1061C000A9010E943632882309F440C0C1E2D1E01F
:1061D00017FF05C0119501951109C9E0D1E06E01C5
:1061E000B8E1CB1AD10880E2E82EF12C0FC0D5011E
:1061F000B1CFFE0125913591459154910E191F099A
:10620000C501B4010E949C324B015C01D501C4015F
:106210000E151F0574F72497F594E794CC16DD0648
:10622000A9F78A2F880F8B2F881F8F3F49F020E016
:1062300030E0A901C501B4010E943632811106C0C7
:1062400082E290E09093450680934406C501B40134
:10625000CDB7DEB7ECE00C94A033283008F027E08F
:106260003327DA01990F311D87FD91600096610592
:10627000710539F432602E5F3D9330E32A95E1F7E2
:1062800008959F3F30F080387105610509F03C5F4B
:106290003C5F3D93913008F08068911DDF93CF9370
:1062A0001F930F93FF92EF92192F987F9695E92FE6
:1062B00096959695E90FFF27E158FE4F99273327CA
:1062C000EE24FF24A701E70105900894079428F421
:1062D000360FE71EF81E491F511D660F771F881FD6
:1062E000991F0694A1F70590079428F4E70EF81E6D
:1062F000491F561FC11D770F881F991F661F0694DF
:10630000A1F70590079428F4F80E491F561FC71FE0
:10631000D11D880F991F661F771F0694A1F705905E
:10632000079420F4490F561FC71FD81F990F661FE7
:10633000771F881F0694A9F784911095177041F074
:10634000D695C79557954795F794E7941A95C1F751
:10635000E5E2F1E06894159015913591659195917C
:1063600005907FE27395E118F10A430B560BC90BB8
:10637000D009C0F7E10CF11E431F561FC91FD01DE5
:106380007EF4703311F48A95E6CFE894015030F032
:10639000080F0AF40027021708F4202F2395022F74
:1063A0007A3328F079E37D932A95E9F710C07D933D
:1063B0002A9589F6069497956795379517951794BA
:1063C000E118F10A430B560BC90BD00998F023953D
:1063D0007E9173957A3308F070E37C932013B8F7BD
:1063E0007E9170617D9330F0839571E37D9370E3CE
:1063F0002A95E1F71124EF90FF900F911F91CF9113
:10640000DF91992787FD9095089591110C94093398
:10641000803219F089508550C8F70895FB01DC01DE
:106420004150504088F08D9181341CF08B350CF434
:10643000805E659161341CF06B350CF4605E861BE8
:10644000611171F3990B0895881BFCCFDC01FC01ED
:10645000672F71917723E1F7329704C07C916D9398
:1064600070836291AE17BF07C8F308950E94783217
:1064700008F481E00895E89409C097FB3EF49095F4
:106480008095709561957F4F8F4F9F4F9923A9F00D
:10649000F92F96E9BB279395F6958795779567959C
:1064A000B795F111F8CFFAF4BB0F11F460FF1BC0E0
:1064B0006F5F7F4F8F4F9F4F16C0882311F096E973
:1064C00011C0772321F09EE8872F762F05C0662321
:1064D00071F096E8862F70E060E02AF09A95660FDA
:1064E000771F881FDAF7880F9695879597F9089593
:1064F000990F0008550FAA0BE0E8FEEF16161706D5
:10650000E807F907C0F012161306E407F50798F03C
:10651000621B730B840B950B39F40A2661F0232B55
:10652000242B252B21F408950A2609F4A140A695D1
:106530008FEF811D811D08950E94AF320C9423338B
:106540000E94153338F00E941C3320F0952311F07F
:106550000C940C330C94123311240C9457330E9476
:10656000343370F3959FC1F3950F50E0551F629F30
:10657000F001729FBB27F00DB11D639FAA27F00D9C
:10658000B11DAA1F649F6627B00DA11D661F829FC3
:106590002227B00DA11D621F739FB00DA11D621FA8
:1065A000839FA00D611D221F749F3327A00D611DC5
:1065B000231F849F600D211D822F762F6A2F1124A7
:1065C0009F5750409AF0F1F088234AF0EE0FFF1FDA
:1065D000BB1F661F771F881F91505040A9F79E3F31
:1065E000510580F00C940C330C9457335F3FE4F367
:1065F000983ED4F3869577956795B795F795E79587
:106600009F5FC1F7FE2B880F911D9695879597F98F
:10661000089599278827089597F99F6780E870E083
:1066200060E008959FEF80EC089500240A94161608
:10663000170618060906089500240A941216130670
:10664000140605060895092E0394000C11F48823FE
:1066500052F0BB0F40F4BF2B11F460FF04C06F5F1A
:106660007F4F8F4F9F4F089557FD9058440F551FF0
:1066700059F05F3F71F04795880F97FB991F61F0C4
:106680009F3F79F087950895121613061406551F3B
:10669000F2CF4695F1DF08C0161617061806991FA7
:1066A000F1CF86957105610508940895E894BB279C
:1066B00066277727CB0197F90895F999FECF92BD08
:1066C00081BDF89A992780B50895262FF999FECFB4
:1066D0001FBA92BD81BD20BD0FB6F894FA9AF99AFF
:1066E0000FBE019608950E94B533A59F900DB49FEB
:1066F000900DA49F800D911D112408952F923F921B
:106700004F925F926F927F928F929F92AF92BF92C1
:10671000CF92DF92EF92FF920F931F93CF93DF936D
:10672000CDB7DEB7CA1BDB0B0FB6F894DEBF0FBECA
:10673000CDBF09942A88398848885F846E847D8417
:106740008C849B84AA84B984C884DF80EE80FD8019
:106750000C811B81AA81B981CE0FD11D0FB6F8948F
:10676000DEBF0FBECDBFED010895A29FB001B39F64
:10677000C001A39F700D811D1124911DB29F700D4A
:10678000811D1124911D08955058BB27AA270E94EE
:10679000DC330C9423330E94153338F00E941C33F1
:1067A00020F039F49F3F19F426F40C9412330EF4C0
:1067B000E095E7FB0C940C33E92F0E94343358F337
:1067C000BA17620773078407950720F079F4A6F5D6
:1067D0000C9456330EF4E0950B2EBA2FA02D0B011E
:1067E000B90190010C01CA01A0011124FF27591B16
:1067F00099F0593F50F4503E68F11A16F040A22F1C
:10680000232F342F4427585FF3CF4695379527958C
:10681000A795F0405395C9F77EF41F16BA0B620B8B
:10682000730B840BBAF09150A1F0FF0FBB1F661FD2
:10683000771F881FC2F70EC0BA0F621F731F841F15
:1068400048F4879577956795B795F7959E3F08F03B
:10685000B0CF9395880F08F09927EE0F97958795FD
:1068600008950E9445340C9423330E941C3358F041
:106870000E94153340F029F45F3F29F00C940C334B
:1068800051110C9457330C9412330E94343368F333
:106890009923B1F3552391F3951B550BBB27AA27D9
:1068A00062177307840738F09F5F5F4F220F331F13
:1068B000441FAA1FA9F335D00E2E3AF0E0E832D0DB
:1068C00091505040E695001CCAF72BD0FE2F29D0DE
:1068D000660F771F881FBB1F261737074807AB07B0
:1068E000B0E809F0BB0B802DBF01FF2793585F4F25
:1068F0003AF09E3F510578F00C940C330C945733CA
:106900005F3FE4F3983ED4F3869577956795B79506
:10691000F7959F5FC9F7880F911D9695879597F911
:106920000895E1E0660F771F881FBB1F621773078A
:106930008407BA0720F0621B730B840BBA0BEE1F9F
:1069400088F7E09508950E94AA346894B1110C94D8
:10695000573308950E943C3388F09F5798F0B92F21
:106960009927B751B0F0E1F0660F771F881F991F84
:106970001AF0BA95C9F714C0B13091F00E9456339D
:10698000B1E008950C945633672F782F8827B85FAD
:1069900039F0B93FCCF3869577956795B395D9F7DC
:1069A0003EF490958095709561957F4F8F4F9F4FE6
:1069B000089597FB16F40E941D350C94E034E8947A
:1069C000F92F96EBFF2381F0121613061406440BE1
:1069D0009395F69587957795679557954040FF2352
:1069E000B9F71BC099270895882351F49850D2F71E
:1069F000872B762F652F542F432F322F20E0B1F3B2
:106A0000121613061406440B88233AF09A95440F85
:106A1000551F661F771F881FCAF755234AF4440F76
:106A2000551F11F460FF04C06F5F7F4F8F4F9F4F62
:106A3000880F9695879597F908959095809570950C
:106A4000609550954095309521953F4F4F4F5F4F42
:106A50006F4F7F4F8F4F9F4F08950E94783208F4F9
:106A60008FEF0895FA01EE0FFF1F309621053105D3
:106A7000A1F16115710561F48038BFE39B0749F10D
:106A800068949038810561F08038BFEF9B0741F032
:106A900099234AF5FF3FE1053105210519F1E894F5
:106AA0000894E795D901AA2329F4AB2FBE2FF85FEC
:106AB000D0F310C0FF5F70F4A695E0F7F73950F0FF
:106AC00019F0FF3A38F49F779F930DD00F9007FC91
:106AD0009058089546F00C94123360E070E080E81E
:106AE0009FE308954FE79F775F934F933F932F93D3
:106AF0000E9432362F913F914F915F910E949C32BC
:106B00000C948F350E947832880B990B089529F4E4
:106B100016F00C940C330C9456330C9412330E94E0
:106B20003C33A8F39638A0F707F80F92E8942BE3CC
:106B30003AEA48EB5FE70E94B2320F920F920F924F
:106B40004DB75EB70F920E947A36E8E6F0E00E94F9
:106B5000C1354F915F91EF91FF91E595EE1FFF1FBA
:106B600049F0FE57E0684427EE0F441FFA95E1F71D
:106B70004195550B0E94F4350F9007FE0C94E835B3
:106B80000895DF93CF931F930F93FF92EF92DF92BD
:106B90007B018C01689406C0DA2EEF010E94AF32AF
:106BA000FE01E894A5912591359145915591A6F363
:106BB000EF010E94DC33FE019701A801DA9469F726
:106BC000DF90EF90FF900F911F91CF91DF9108958B
:106BD0009B01AC0160E070E080E89FE30C943134ED
:106BE0000C940C330C94AE360E943C33D8F39923AA
:106BF000C9F3940F511DA3F39150504094F059F0F4
:106C0000882332F0660F771F881F91505040C1F7DC
:106C10009E3F51052CF7880F911D9695879597F902
:106C200008955F3FACF0983E9CF0BB278695779522
:106C30006795B79508F4B1609395C1F7BB0F58F706
:106C400011F460FFE8CF6F5F7F4F8F4F9F4FE3CF0F
:106C50000C94573316F00C94AE360C94123368949F
:106C60000C940C330E943C33A8F39923C1F3AEF388
:106C7000DF93CF931F930F93FF92C92FDD278823B4
:106C80002AF02197660F771F881FDAF720E030E09F
:106C900040E85FEB9FE3883920F0803E38F0219692
:106CA0008F770E94C533E0E9F0E004C00E94C5334D
:106CB000EDEBF0E00E94C1358B01BE01EC01FB2E33
:106CC0006F5771097595771F880B990B0E943D329C
:106CD00028E132E741E35FE30E94AF32AF2D980134
:106CE000AE01FF900F911F91CF91DF910E94DC3395
:106CF0000C942333FA01DC01AA0FBB1F9B01AC01EA
:106D0000BF5728F4222733274427507820C0B75193
:106D100090F4AB2F0024469537952795011CA39539
:106D2000D2F3002071F0220F331F441FB395DAF322
:106D30000ED00C94C43361307105A0E88A07B946BF
:106D400030F49B01AC01662777278827907830962E
:106D500021F0208331834283538308959F3F31F094
:106D6000915020F4879577956795B795880F911D79
:106D70009695879597F90895DB018F939F930E94CD
:106D80007333BF91AF91A29F800D911DA39F900D72
:106D9000B29F900D11240895AA1BBB1B51E107C09F
:106DA000AA1FBB1FA617B70710F0A61BB70B881F9B
:106DB000991F5A95A9F780959095BC01CD0108952A
:106DC00097FB072E16F4009407D077FD09D00E9498
:106DD000CC3607FC05D03EF4909581959F4F0895E1
:106DE000709561957F4F0895A1E21A2EAA1BBB1BD7
:106DF000FD010DC0AA1FBB1FEE1FFF1FA217B30787
:106E0000E407F50720F0A21BB30BE40BF50B661F9C
:106E1000771F881F991F1A9469F760957095809560
:106E200090959B01AC01BD01CF010895052E97FB04
:106E30001EF400940E942D3757FD07D00E94F436AF
:106E400007FC03D04EF40C942D37509540953095A7
:106E500021953F4F4F4F5F4F0895909580957095C6
:106E600061957F4F8F4F9F4F0895EE0FFF1F059045
:106E7000F491E02D0994B7FF0C9473330E9473339F
:106E8000821B930B0895DF93CF931F930F939A9DCB
:106E9000F02D219FF00D8B9DF00D8A9DE02DF10DC1
:106EA000039FF00D029FE00DF11D4E9DE00DF11DC1
:106EB0005E9DF00D4F9DF00D7F936F93BF92AF924B
:106EC0005F934F93D5010E94B5338B01AC01D7017D
:106ED0000E94B533EB01E80FF91FD6010E949237EB
:106EE0002F913F91D6010E94B533C60FD71FE81FDF
:106EF000F91FAF91BF910E9492372F913F910E944D
:106F0000B533C60FD71FE81FF91FD6010E94B5334E
:106F1000E60FF71F9801BE01CF010F911F91CF918E
:106F2000DF9108950E94B533460F571FC81FD91F20
:106F300008F431960895689401C0E894F92FF12B74
:106F400012F00C94CF37A0E0B0E0E9EAF7E30C943C
:106F50008433092E059422F40E942B38112392F4D5
:106F6000F0E80F26FFEFE094F09400951095B094B0
:106F7000C094D094A194BF0ACF0ADF0AEF0AFF0A97
:106F80000F0B1F0B0E94DA3707FC0E942B38CDB77E
:106F9000DEB7ECE00C94A033689401C0E8948F92C3
:106FA0009F92CF93DF930E94DA37DF91CF919F902A
:106FB0008F90089588249924F401E401B0E49F930C
:106FC000AA279A158B049C04ED05FE05CF05D00772
:106FD000A10798F4AD2FDC2FCF2FFE2FE92D982C91
:106FE000892E982F872F762F652F542F432F322FDE
:106FF0002227B85031F7BF9127C01B2EBF91BB2766
:10700000220F331F441F551F661F771F881F991FAC
:10701000881C991CEE1FFF1FCC1FDD1FAA1FBB1F62
:107020008A149B04EC05FD05CE05DF05A007B1071A
:1070300048F08A189B08EC09FD09CE09DF09A00B6E
:10704000B10B21601A94E1F62EF49401AF01BE0158
:10705000CD01000C089560957095809590953095C0
:107060004095509521953F4F4F4F5F4F6F4F7F4F4A
:107070008F4F9F4F0895002E083090F0982F872F44
:10708000762F652F542F432F322F22270850F4CF0D
:10709000220F331F441F551F661F771F881F991F1C
:1070A0000A95B2F7002D089597FD1094002E083030
:1070B00098F00850232F342F452F562F672F782F05
:1070C000892F912DF4CF159497958795779567958E
:1070D00057954795379527950A95AAF71124002DBE
:1070E00008952A0D3B1D4C1D5D1D6E1D7F1D801FCB
:1070F000911F08952A193B094C095D096E097F0902
:10710000800B910B08950024A7FD00942A173005E9
:1071100040055005600570058005900508950F93A2
:107120001F93CF93DF938230910510F482E090E0BB
:10713000E0914806F091490630E020E0B0E0A0E0A0
:10714000309799F42115310509F44AC0281B390BF1
:1071500024303105D8F58A819B816115710589F14B
:10716000FB0193838283FE0111C040815181028122
:10717000138148175907E0F04817590799F41097F9
:1071800061F012960C93129713961C933296CF01CE
:10719000DF91CF911F910F910895009348061093AE
:1071A0004906F4CF2115310551F04217530738F045
:1071B000A901DB019A01BD01DF01F801C1CFEF0197
:1071C000F9CF9093490680934806CDCFFE01E20F98
:1071D000F31F819391932250310939832883D7CFAC
:1071E0002091460630914706232B41F4209124013B
:1071F00030912501309347062093460620912201C5
:10720000309123012115310541F42DB73EB740914E
:10721000260150912701241B350BE0914606F09181
:107220004706E217F307A0F42E1B3F0B2817390778
:1072300078F0AC014E5F5F4F2417350748F04E0FD2
:107240005F1F5093470640934606819391939FCFCB
:10725000F0E0E0E09CCFCF93DF930097E9F0FC01F2
:10726000329713821282A0914806B0914906ED012F
:1072700030E020E01097A1F420813181820F931F2C
:1072800020914606309147062817390709F061C05A
:10729000F0934706E0934606DF91CF910895EA0107
:1072A000CE17DF07E8F54A815B819E014115510544
:1072B000B1F7E901FB83EA8349915991C40FD51FC6
:1072C000EC17FD0761F4808191810296840F951F70
:1072D000E90199838883828193819B838A83F0E08B
:1072E000E0E012968D919C9113970097B9F52D913E
:1072F0003C911197CD010296820F931F2091460673
:10730000309147062817390739F6309751F5109212
:10731000490610924806B0934706A0934606BCCF94
:10732000D383C28340815181840F951FC817D90729
:1073300061F44E5F5F4F88819981480F591F5183D7
:1073400040838A819B81938382832115310509F0D3
:10735000B0CFF0934906E09348069ECFFD01DC01D3
:10736000C0CF13821282D7CFB0E0A0E0EAEBF9E3FE
:107370000C9480338C01009751F4CB010E948F381C
:107380008C01C801CDB7DEB7E0E10C949C33FC0161
:10739000E60FF71F9C0122503109E217F30708F4AA
:1073A0009DC0D901CD91DC911197C617D70798F0F0
:1073B000C530D10530F3CE0104978617970708F33F
:1073C000C61BD70B2297C193D1936D937C93CF01AA
:1073D0000E942B39D6CF5B01AC1ABD0A4C018C0E32
:1073E0009D1EA0914806B0914906512C412CF12CCC
:1073F000E12C109731F5809146069091470688154B
:10740000990509F05CC04616570608F058C08091EF
:10741000220190912301009741F48DB79EB74091CE
:10742000260150912701841B950BE817F90708F0F6
:1074300055C0F0934706E0934606F90171836083D7
:10744000A0CF8D919C91119712966C9012971396E4
:107450007C901397A815B90559F56C0142E0C40E4C
:10746000D11CCA14DB0420F1AC014A195B09DA0112
:107470001296159780F06282738251834083D901FE
:107480006D937C93E114F10471F0D7011396FC9392
:10749000EE93129776CF22968C0F9D1FF901918360
:1074A0008083F301EFCFF0934906E093480669CF5C
:1074B0004816590608F42C017D01D3019ACFCB015F
:1074C0000E948F387C01009749F0AE01B8010E94FC
:1074D000793AC8010E942B39870153CF10E000E0B0
:1074E00050CF9111089581568A5108F480528558E1
:1074F0000895FB01DC0102C001900D924150504003
:10750000D8F70895FB01DC0101900D920020E1F70E
:107510000895FB01DC014150504030F08D91019005
:10752000801919F40020B9F7881B990B0895FB0105
:10753000DC014150504048F001900D920020C9F705
:1075400001C01D9241505040E0F70895FB01519158
:107550005523A9F0BF01DC014D9145174111E1F719
:1075600059F4CD010190002049F04D914015411191
:10757000C9F3FB014111EFCF81E090E0019708953D
:1075800013E0C1E7D3E004C0FE010E943537219625
:10759000C237D107C9F7F894FFCF08200000008058
:1075A00004030000A040C800017F0A0000000001A1
:1075B00064000000F041A80E0001D10D00004A0651
:1075C00080005E00BC007701000100FF0100FF00A9
:1075D000000000009904E0032604E6045704350483
:1075E000490400000000500A230AE60FF9091C0AAA
:1075F000090AFA0900000000BF0FE003E60FDF03ED
:107600000D0A0020202020202020202020202020C3
:107610002000524542005645520023566572736958
:107620006F6E3A004C4F4700234C6F6767657220BE
:107630004E616D653A0053484F57533D00474554DE
:1076400000732000534156453D0054494D45493D86
:107650000023496E74657276616C3D0054494D4556
:10766000443D00234475726174696F6E3D0042545D
:107670003D00534C20503D00506120756E6C696B8D
:10768000656C792100685061004E45543D005556A7
:107690005A002355562056303D005620004D533D8C
:1076A000002C0023496E636F727265637421204D54
:1076B000533D31323344334435005428312C322C7D
:1076C00033293D00445354286F432900206F432041
:1076D000445320546865726D6F6D65746572002047
:1076E000572F6D5E3200555620496E74656E736972
:1076F000747900572F6D5E32200055563D0068505A
:107700006120006F43006D0020413D00495220463A
:107710006C616D65204C6576656C3D00476173203A
:107720006C6576656C3D00204D756C746973656E93
:10773000736F72730023456E61626C650023446948
:107740007361626C650044440023496E76616C6924
:1077500064206B65792100424E4D4C3033006E61E0
:107760006E6F424432693744535400234E6F2053A6
:10777000656E736F72210057656C636F6D653A00BB
:1077800023626D70206661696C656400736572695F
:0E779000616C3A20002D35002D34002D3300A1
:107E0000112484B714BE81FFF0D085E080938100F7
:107E100082E08093C00088E18093C10086E0809377
:107E2000C20080E18093C4008EE0C9D0259A86E02C
:107E300020E33CEF91E0309385002093840096BBD3
:107E4000B09BFECF1D9AA8958150A9F7CC24DD24C4
:107E500088248394B5E0AB2EA1E19A2EF3E0BF2EE7
:107E6000A2D0813461F49FD0082FAFD0023811F036
:107E7000013811F484E001C083E08DD089C08234E0
:107E800011F484E103C0853419F485E0A6D080C0E4
:107E9000853579F488D0E82EFF2485D0082F10E0AE
:107EA000102F00270E291F29000F111F8ED06801E7
:107EB0006FC0863521F484E090D080E0DECF843638
:107EC00009F040C070D06FD0082F6DD080E0C81688
:107ED00080E7D80618F4F601B7BEE895C0E0D1E017
:107EE00062D089930C17E1F7F0E0CF16F0E7DF06D8
:107EF00018F0F601B7BEE89568D007B600FCFDCFD4
:107F0000A601A0E0B1E02C9130E011968C91119780
:107F100090E0982F8827822B932B1296FA010C0160
:107F200087BEE89511244E5F5F4FF1E0A038BF0790
:107F300051F7F601A7BEE89507B600FCFDCF97BE46
:107F4000E89526C08437B1F42ED02DD0F82E2BD052
:107F50003CD0F601EF2C8F010F5F1F4F84911BD097
:107F6000EA94F801C1F70894C11CD11CFA94CF0C13
:107F7000D11C0EC0853739F428D08EE10CD085E9AC
:107F80000AD08FE07ACF813511F488E018D01DD067
:107F900080E101D065CF982F8091C00085FFFCCF94
:107FA0009093C60008958091C00087FFFCCF809118
:107FB000C00084FD01C0A8958091C6000895E0E648
:107FC000F0E098E1908380830895EDDF803219F02E
:107FD00088E0F5DFFFCF84E1DECF1F93182FE3DFCA
:107FE0001150E9F7F2DF1F91089580E0E8DFEE27F6
:047FF000FF270994CA
:027FFE00040479
:00000001FF
